:10000000980B0020E5000000C1000000C1000000C6
:1000100000000000000000000000000000000000E0
:10002000000000000000000000000000C10000000F
:100030000000000000000000C1000000C10000003E
:10004000012D0000C5050000452E00004D220000D6
:10005000CD21000001220000652500002D260000B2
:10006000C1000000C9010000E90100000902000010
:10007000FD060000E5450000C1000000C1000000D1
:10008000C1000000C1000000C1000000C10000006C
:10009000C1000000C1000000C1000000C10000005C
:1000A000C1000000C1000000C1000000C10000004C
:1000B0006D2D0000616B0000C1000000C100000058
:1000C000A02130B559251624054AC90588230120E9
:1000D0005560546053608B6803438B60F6E7C046FD
:1000E000FC000050002370B50A480B490B4C1A184D
:1000F0008A4203D2E55804331560F8E70021084B23
:10010000084A934201D202C3FBE704F0DFFD00F08E
:1001100021FE70BD0000002000010020546F00008F
:100120000001002094070020002307B50193032855
:100130001DD8114B02301A6880000723C2401A40B4
:100140006B4603331A701A78002A02D102F01EFEA1
:1001500004E01A78022A03D102F04EFE019004E076
:100160001B78072B05D1054B0193019802E0044849
:1001700000E004480EBDC04614020050008051014A
:100180000197FFFF0297FFFFF8B507000E00012857
:1001900015D9002913D001240D002900380006F0DC
:1001A0003FFD084A831E934203D8013C24062043A6
:1001B00007E080230134AD195B009C42EDD10120A2
:1001C0004042F8BDFDFFFF00012110B5044A9368CD
:1001D0000B439360034BDA681869904710BDC04623
:1001E0002000014000010020012110B5044A93685D
:1001F0000B439360034B1A6A586A904710BDC04680
:100200000000114000010020012110B50C4A0D4CE6
:1002100093680B439360A36A5B18A362E36A002BA5
:100220000CD0236B002B09D0A36B013BA363002BE5
:1002300004D1E36B206C9847636BA36310BDC04689
:1002400020001140000100200122034B5A649A64EF
:10025000DA641A657047C04600010020F7B50C004B
:100260000190009203287DD8414B06F0C5FC021F87
:100270003D54596C012977D1586D002874D1042759
:100280003C4E5965B2683A43B2603B4E3060B2684A
:100290000A43B260D86698651C67FFF745FF2100E6
:1002A000FFF772FF431C4DD1344860E0986C012881
:1002B0005AD15A6F002A57D108272E4E5867B16875
:1002C0003943B1602E4E3260B1680143B1601A60AB
:1002D0009A67DC67FFF728FF2100FFF755FF431CF3
:1002E000E2D00302FB402FE0D86C01283CD1254A24
:1002F0001168002938D110251E4F1060BE682E43AA
:10030000BE60214E3160B7683843B06051605961BA
:1003100094600220C1E7186D012825D11949CA68E7
:10032000002A21D12025134FC860BE682E43BE602D
:10033000164E3260B7683843B0609A621A630C6137
:100340000320AAE703021B0A7360009B000EDB0672
:100350001843009B3060022B08D101980F30C0B2C7
:1003600002F00EF80A4802E00A4800E00020FEBD54
:100370000001002000020050000001400297FFFF32
:1003800020000140800100200000114020001140A9
:100390000197FFFF0397FFFF73B50024032800D9DF
:1003A000C4E0634C06F028FC023262916569002DBE
:1003B00000D0BAE001201426A061606901306061BC
:1003C0005C4C0195019800282FDC019D1420754399
:1003D0006519AD6D002D15D10126019D45436519A7
:1003E000AE65019D45436519E965019D4543651964
:1003F00029660199414361184A66019A50432018C1
:10040000836690E0019801300190DBE7E569002DFB
:1004100000D08AE0012014262062E0690130E0610A
:10042000444C01950198002801DD00247EE0019DE7
:10043000142075432D59002D14D10126019D4543EB
:100440006651019D454365196960019D45436519E4
:10045000A960019941436118CA60019A504320186C
:10046000036160E0019801300190DBE7656A002DCF
:100470005BD101201426A062606A013060622D4CBD
:10048000019501980028D0DC019D14207543651961
:100490006D69002D15D10126019D454365196E61D9
:1004A000019D45436519A961019D45436519E961B0
:1004B0000199414361180A62019A5043201843622E
:1004C00031E0019801300190DBE7E66A002E2CD183
:1004D00001251848C562E56A0135E56201961436C2
:1004E00002E0019C01340194019C002C9DDC019DE3
:1004F0001424754345192D6B002DF2D10126019D61
:10050000654345192E63019D654345196963019D46
:1005100065434519A963019961434118CA63019A6A
:10052000544300190364019C00E0034C200076BD95
:1005300080010020000100200497FFFF30B5032850
:100540001FD88021104B8200D358104A89059B1870
:100550001A6808300A431A600323FF22C0B2C2247B
:100560000340DB009A400A49A4000D5995438022BC
:100570009A4013002B430B510123834000200B6052
:1005800000E0044830BDC0460C6F00000000014090
:1005900000E100E00197FFFF03280BD88021064B04
:1005A0008000C358054AC9059B181A6800200A43F1
:1005B0001A6000E0024870470C6F00000000014024
:1005C0000197FFFF07B50821074A13689B06DB0F59
:1005D000019313680B431360044B1B6B002B01D07A
:1005E0000198984707BDC0460040004080010020A8
:1005F00010B501240C4B5B68234213D080230B49B8
:100600008A6822438A600A4A116899431160146813
:10061000793B184003022000064908401843106047
:10062000002000E0044810BDFC0000500002005013
:1006300000400040FFF8FFFF0697FFFF4021034AFC
:1006400013680B431360024B18637047004000406F
:100650008001002000B5092842D8224B06F0CCFAD0
:1006600005080B1C24282B2E31371A6880211DE029
:100670001A68802127E040211A680A43C0211A60C5
:10068000194A89005058194B034080200002034347
:1006900053500223136018E040211A688A431A60FD
:1006A0000222134BDA6710E010211A680A430BE0AC
:1006B0001A68102107E01A680121F7E71A68022179
:1006C000F4E702211A688A431A60002009E0072231
:1006D000114018680A020749014011431960F4E704
:1006E000054800BD0040004000E100E0FF00FFFFC2
:1006F00004E100E0FFF8FFFF0597FFFF044B10B592
:100700001868044B1B68002B00D0984710BDC046EA
:100710001C000540B4010020824BF7B50D001842C3
:1007200000D0F3E08A79072A00D9F1E0AB23D34067
:10073000DB0700D4ECE00B79032B00D9EAE04B791E
:10074000012B00D9E8E0CB79062B00D9E6E0A02305
:10075000DB057549DA688024002805D1640222434C
:10076000DA60DE68714A04E0A4022243DA60DE68DF
:100770006F4A3240DA608B680F2623438B606D4BE3
:10078000C4180420A3680343A3600223A2681A4389
:10079000A260EF79A2683E40F0278640BA43324318
:1007A000A260AE79D03F0640721E9641E2687601A3
:1007B000BA433243E260AA79E76813405A1E934174
:1007C0001A0110239F433B00012608271343E360CF
:1007D000AA79E3683240D200BB431343E360E36885
:1007E0002A79053F3A40BB431343E360E2686B79E3
:1007F00082431E40B30016001E43E660236A2A7A35
:10080000FB308343134323620A68474BD20703D567
:100810005869494A02400FE01A6AD20305D4586960
:10082000454A02408020400405E01A68520777D507
:10083000C0205A69800402435A618E694B693605AB
:10084000360F9B019B0F0136002B02D102F09EFA5E
:1008500007E0354B5B699B019B0F012B03D102F035
:1008600099FA310001E03100344806F0D9F92F68D7
:100870000600390006F0D4F90F2305000340626A30
:10088000012B0CD87F01B74209D22D4B050913402B
:100890006362626A2B4BAF1E134063622EE08021BD
:1008A000802389050A436262626A5B051A43264B0C
:1008B000AF1E62629F4221DD0826636A0B436362BA
:1008C000626A204B13406362731C19002800019375
:1008D00006F02CFA02290ED80F23616A1B4A1E402B
:1008E000114033060E001E4366620199280006F08F
:1008F00097F9871E02E0019E102EE5D1656AB8B215
:100900002D0C2D040543656200200AE0104808E024
:10091000104806E0104804E0104802E0104800E0EB
:100920001048FEBDFFFFEFFF00020050FFFFFEFF7B
:10093000FFFFFDFF00000540FFFFFFFC00805101AD
:10094000FFFFFFDFFFFFFFEFFFFF0000FFFFFFF0F4
:100950000298FFFF0398FFFF0498FFFF0598FFFF31
:100960000698FFFF0898FFFFF7B501240E002E4BF5
:100970000192C3185D682640A54335434E080227FF
:100980002640A6405D605D68BD4335438E08264025
:10099000BE405D605D68FF19BD4335435D605D68C5
:1009A000CE0826400437F600BD4335435D605E68DF
:1009B0000D09B44662461D4E2540EF0216403E43E7
:1009C00010275E605E682D01BE4335434E098909DC
:1009D00026400C40A10140245D605D68FF1976014E
:1009E000BD4335435D605D68A5432C000C43C321C6
:1009F0005C6089000E4B00280BD1019A0D48026003
:100A0000FF205A5882437F3802435A5080225201B5
:100A100008E05858084A02408020000202435A5019
:100A2000802292011A60F7BD00000540FFF7FFFF2A
:100A300000E100E0B4010020FF00FFFF0322F0B559
:100A4000214B224EC018036B214F134303634C7894
:100A50000123621E9441C56A1E4AE4032A402243D0
:100A6000C262C56A8A7814062A02120A2243C26246
:100A70000C78C26A1C40324024022243C2620C78C5
:100A8000C26ADC40144D1C4064022A402243C26208
:100A90000C78C26AA4081C40A4023A402243C262F5
:100AA000076ACC780D4A24023A40224302620A794E
:100AB000816813401A020B003340134383600369BB
:100AC0001D400561F0BDC04600000540FFFEFFFF70
:100AD000FFFBFFFFFF7FFFFFFFFDFFFFFF00FFFFAB
:100AE00030B50F240125124BDA68A2432A43DA609D
:100AF000DA686419A243DA602022DC681443DC60FF
:100B0000586099601A692A431A61BFF36F8F186998
:100B1000074AC007C00FC0B20028F8D113685B06AF
:100B200004D54021136803480B43136030BDC04611
:100B300000C000508188FFFF10B50F24134BDA6806
:100B4000A243DA60DA680134A243DA60DA6810346A
:100B5000A243DA600022586001209A601A690243B9
:100B60001A61BFF36F8F1869084AC007C00FC0B27F
:100B70000028F8D113685B0605D5402113680448A6
:100B80000B43136001E093680B6010BD00C0005080
:100B90008188FFFF0F21124BDA688A430D390A431F
:100BA000DA60DA680E318A43DA60DA6810310A43B3
:100BB000DA6058601A691F390A431A61BFF36F8FF0
:100BC0001869074AC007C00FC0B20028F8D11368DF
:100BD0005B0604D54021136802480B43136070473D
:100BE00000C000508188FFFF0421054A53680B4371
:100BF0005360044A033913680B4313607047C046BF
:100C00000002005000C000500121024A13688B43CB
:100C10001360704700C0005010B516205924882179
:100C2000034B5C60586059605A68002AF9D010BDC7
:100C3000FC000050F0B50C0085B0FF2813D1022154
:100C40003D4A93680B439360FFF7E6FFFFF7CCFF45
:100C5000F8204002FFF79EFFA0220121D2059368F1
:100C60000B439360FEE70130C5B2FF20152D60D81D
:100C7000012D0ED1092905D90B1C182900D91823DB
:100C8000DCB200E00A242D4B1B190A3B1A782C4BCE
:100C90001A602C4B585D0193C0B2844249D0FFF7D3
:100CA000BBFF8022284B9201DA67FFF79DFFF823F4
:100CB000DB01EE18B60003A93000FFF73DFF039BF0
:100CC000102723409C4209D1204B3000E1180391AA
:100CD000FFF706FF1EE0013F002F1BD0F820400267
:100CE000FFF758FFF82003A94002FFF725FF039BF9
:100CF0000133F0D1019B5C550024019B195D134B1E
:100D0000C918F823DB01E01880000134FFF7E8FE82
:100D1000152CF2D103A93000FFF70EFF039BDCB2C4
:100D2000FFF772FF80220A4B92011A6001F0D2FF96
:100D3000200005B0F0BDC046004100501C6F00000F
:100D400010000440E702002004E100E00000FFFF83
:100D500000E100E0F0B5594B594F5A4A3B605A4BFD
:100D60005A4E1A605A4A5B4D32605B4A5B4C2A60AD
:100D70005B4AF9B022608022B2600022BA609A60B9
:100D80000A23AB602E33A360FFF746FF0121554BCA
:100D90001A680A431A6008971F000396059507947E
:100DA000FB68504ADB07FBD5116A4F4B4F4C0B4099
:100DB00013620C2301212360BC3322681A430A42C8
:100DC00004D122685B0852082260F6E7C02122683D
:100DD0000902023A5202386A0A43023B1343DA0517
:100DE000400A4002D20D02433A62F8229201386A68
:100DF00013403F4A024013433B623B6A1943396246
:100E00003A6A3C4B13403B623B6A3B4A13403B62AD
:100E10000E92FB68334A5B07FBD5072113698B43AE
:100E200005390B431361D3681B0603D5D3687E31A4
:100E30000B43D36003F006FF01F0ACFF2060FFF727
:100E4000D3FEF82012A94002FFF776FE2B4B129A30
:100E50002B4C9A4211D10025F823DB01E8188000C1
:100E600012A9FFF769FE129BDBB263550135152D00
:100E7000F2D1F925234E6D024CE012A92248FFF76A
:100E80005BFEF820129B4002DBB223750025FFF7C2
:100E900081FE142D03D01D4B0F33EB5C6355615D58
:100EA0001B4BC918F823DB01E818800001351291AB
:100EB000FFF716FE152DECD1DBE7C046FFCF000093
:100EC00000400050F0FF00004040005080400050C3
:100ED000FFF70000C0400050CF5D0000004100500F
:100EE000D50F000000020050FFFFF7FFCC020020EA
:100EF000FFC1FFFFFFFFFBFFFFFFFEFFA500FFFF9E
:100F0000E70200204B05002050F001001C6F00009C
:100F10000000FFFF12A92800FFF70EFEF54B129A02
:100F2000E918F54B100E5854110C3170B270110ABB
:100F3000F24A0435717004369542EBD11A78FF2AD3
:100F400003D1DF3A1A7000225A7012A9EC48FFF759
:100F5000F3FDFFF759FE002092210126E94BEA4AF2
:100F60001870129B09061B021B0A13601368E74DD9
:100F70005B181360E64B83221E700323022100934B
:100F8000030005F091FD6A6AE24B13408022920053
:100F900013436B62E04B1E6005F01CFE059B1B6952
:100FA00002959B0701D404232371079B1B691B0730
:100FB00003D40422637993436371079B1B69DB06A7
:100FC00007D408226379134363716379043A934326
:100FD0006371079B1B699B0607D4082263799343BF
:100FE00063716379043A1343637163791B0705D511
:100FF0004022039B9B681343039A93609022002531
:10100000039BA0249B68E4051343039AC34E93609B
:10101000C34BC44A1D70C44B1D70BB4B1B68DBB275
:101020001370C24A13701F2311780B401370C04A0B
:10103000C04B11680B4003210B431360BE4ABF4BEA
:1010400011680B40C02109010B4380211360E26845
:1010500049020A43E260E2680E9B1A40E260BB6804
:101060000B430421BB60B64B9A680A439A609A68A6
:1010700002390A439A609A68EE318A439A60DA68C4
:10108000D0398A43DA60DA681D390A43DA60DA68EF
:1010900001318A43DA60DA688A43DA601A6AFB311E
:1010A0008A431A627A69A74B13407B61BB691B05AF
:1010B0001B0F049301F06AFE8022336892051343EC
:1010C000802233603368520513433360049B591CFC
:1010D00005F0A6FD9C4905F0A3FD3268023883B2F5
:1010E000100C000418433060226B984BC326134049
:1010F00008222363236B012193432363236B944AC8
:10110000280013402363236BB60013402363914AE6
:10111000FFF72AFCFF22904C1420A35993437F3AF7
:101120001343A35101F02CF98C498D4B0A220B601B
:1011300003230B71012380204D718B71724BCD7194
:101140001B6840031343DBB20B72FFF7E5FA012380
:1011500010A980204B70052340030B708D70CD705B
:101160000D71FFF76BFC80202A0001214003FFF77F
:10117000FBFBA3597B4A290013408022D201134371
:10118000A351062001F088F80221032001F06CF839
:101190000321080001F068F8734B0D201D7001F069
:1011A000EFF80E2001F0ECF8059A704B0C3ED3617D
:1011B0000523059A5B42936109332360A3596C4A66
:1011C00001211340A3512A006A4B032001F080F84B
:1011D000C022A35912061B021B0A1343A35101F09C
:1011E00089FA152001F0CCF8012314AE3370624B5C
:1011F000290015933223280016937570179501F076
:101200003BFD3100280001F0E7FA0121280001F040
:10121000E9FC0121280001F085FA4D4B574A51782D
:101220000F93534B04940693534B0B932B000929B4
:1012300006D951780E33182902D853780A3BDBB20D
:1012400000244F4A0125D25C4E4B4F4E1A604F4B43
:101250001C70FEF7F9FF2022BB684D491343C022E2
:10126000BB603460B36880202B43B3607160336827
:10127000520594461343042233603368C005034388
:101280003360BB681343BB60424B1C609A682A43BF
:101290009A6062465960196811431960FA211A6808
:1012A000890002431A6028002A00FEF7D7FF2800B1
:1012B000FFF772F92800FFF741F92300364A2900A9
:1012C0002800FFF769F8C222049B92009B58254A28
:1012D000C2211340C02212021343049A89005350C2
:1012E000022022002D49FEF7B9FF0220FFF726F960
:1012F00056E0C046000EFEFF4A05002018F201002D
:10130000FC0F1000AC020020B402002000000E40D0
:1013100012030020FFFCFFFF1C00005024000540CA
:101320009007002040050020B00200203904002072
:101330003C000050FCFCFFFF30000050F3F3FFFFC7
:1013400000000540FFFFFFFC90D00300FFF7FFFF08
:10135000FFFBFFFF3145000000E100E0D00200206C
:1013600020A10700FF00FFFF6E050020040004001D
:10137000FFFF00FF8532000030750000E70200200B
:101380001C6F000010000440200011407205002076
:10139000FFFF0000000001406D330000F82A00004C
:1013A0002300C94A29000220FEF7F6FFC222049B4F
:1013B00092009B58C54AC2211340C0221204134315
:1013C000049A890053502000290001F0A9FC03224F
:1013D0007B69062013437B61FFF70AF9BC48FFF7DE
:1013E0002DF921000220FFF735F921002000FFF739
:1013F00031F901F06FFCB74B09961C70B64B1C809D
:10140000B64B1B78A34204D08023B54A1370B54B6A
:101410001D70002301270A930C93049380330693D5
:10142000FFF7FAFBB04A13683B43136001F052FC2C
:10143000AB4B1B785BB2002B03DBFA22AB4B5200A9
:101440001A60AB4B1B685B0728D5FFF7E5FBFFF77E
:10145000CBFBF920F9244002FFF79CFBA54D640269
:10146000A54BA64AE318D15C2B7809061B04C918C2
:101470006B7820001B02C918AB780434C918FFF739
:101480002FFB9F4B04359C42EAD1FFF7BDFB01F0D7
:1014900021FC0421964A13688B431360994B1A6808
:1014A000920541D51968984A0A401A608C4A9749B2
:1014B000127852B2002A01DA052200E000220A70F6
:1014C0000021934A934C11801B682178C9B29B027A
:1014D00011D408250A20FFF7ADFB23788E4CDBB230
:1014E0008E4EE37231780B202943FFF7A3FB33784C
:1014F0001D43257313E008260C20FFF79BFB237880
:10150000854D864CDBB26B7323780D20BB43237073
:1015100021783143FFF78EFB23781E43AE73794A5F
:101520007F4B11680B4013607E4B1B78032B00D060
:101530001EE27D4B1A787D4B1B789A4258D180234E
:1015400070499B040C681C4054D1694B1A685203C3
:1015500050D51A683A424DD01A68BA431A60744B93
:101560001B78002B46D0802206250B68D20413433B
:101570000B60704B1878C0B2421CD2B21A706E4A1F
:1015800015541878C0B2451CEDB21D7005251554D0
:101590001878C0B2451CEDB21D7014541878C0B252
:1015A000441CE4B21C70654CA44666462478E4B240
:1015B000651CEDB2357014541878C0B2441CE4B206
:1015C0001C70862414541878C0B2441CE4B21C70F9
:1015D000042414541878C0B2441CE4B21C70544B58
:1015E0001B78DBB213540A68554B13400B6001E0C3
:1015F00003F0BAFB3E4B1B685B0300D431E1802251
:10160000404BD2041968114000D02AE11A68120236
:1016100000D4EBE018684B4A02401A60304B1B784C
:101620005BB2002B00DB91E020220A24039B434E97
:101630009B689343039A93603E4B1878C0B2421C58
:10164000D2B21A703C4A14541878C0B2441CE4B2A6
:101650001C70092414541878C0B2441CE4B21C70E5
:1016600011541878C0B2441CE4B21C703478E4B24F
:10167000651CEDB23570145418783025C0B2441C86
:10168000E4B21C70B22414541878C0B2441CE4B202
:101690001C7017541878C0B2441CE4B21C706C461D
:1016A0006419247814541878C0B2441CE4B21C7035
:1016B00011541978C9B2481CC0B218702248007879
:1016C000C0B2505483E0C04695390000FFFF00FFD0
:1016D000394C000022030020700500201203002076
:1016E000720500206205002000400040DC0200205E
:1016F0007C0700204B050020000EFEFF4A0500205D
:1017000018F2010068050020FFFDFFFFAC02002079
:10171000AE02002023030020E7020020780700200B
:10172000FFFFCFAF90070020910700208407002023
:1017300080070020E60200203B0400203C0500203A
:10174000FFFFFFFBFFFF7FFF110300200A24BC4BBC
:10175000BC4E1878C0B2421CD2B21A70BA4A1454A5
:101760001878C0B2441CE4B21C70092414541878D0
:10177000C0B2441CE4B21C7011541878C0B2441CAE
:10178000E4B21C703478E4B2651CEDB235701454C8
:101790001878C0B2441CE4B21C70B22414541878F7
:1017A000C0B2441CE4B21C7017541878C0B2441C78
:1017B000E4B21C7011541878C0B2441CE4B21C701E
:1017C00011541878C0B2441CE4B21C70115419783A
:1017D000C9B2481CC0B21870022050541978C9B25E
:1017E000481CC0B218706B461B7C5354974B1A6848
:1017F000520136D505201968954A924D0A401A6063
:101800008F4B1978C9B24A1CD2B21A708E4A505402
:101810001978C9B2481CC0B2187004205054197805
:10182000C9B2481CC0B21870002050541978C9B20F
:10183000481CC0B218702878C0B2441CE4B22C70A6
:1018400050541978C9B2481CC0B21870B020505416
:101850001978C9B2481CC0B218707E4B1B78DBB235
:1018600053547C48069A03789A4200D1BFE003782B
:10187000764A5BB2002B47DB0378DBB20693136832
:101880005B0300D4B3E0802205257349D2040B68C2
:1018900013430B606A4B1C78E4B2621CD2B21A701C
:1018A000694A15551C78E4B2651CEDB21D7004251B
:1018B00015551C78E4B2651CEDB21D700025155558
:1018C0001C78E4B2651CEDB21D705E4D0D94AC4603
:1018D00064462D78EDB26E1CF6B226700D9C15553F
:1018E0001C78E4B2651CEDB21D70B02515551C784E
:1018F000E4B2651CEDB21D700378DBB213550A68C3
:10190000534B13400B6072E02021039B40249B68E3
:101910008B4303998B608021099BC9041B680B438F
:1019200009990B608021099BC9051B680B43099924
:101930000B608021089B9B680B4308998B60059B7B
:1019400005999B68A3438B60444BD978444B49006D
:101950001980FA211368490023431360414B196031
:1019600000231C0018A95C520233802BFAD183E7B4
:10197000384A06991378994239D013785BB2002B14
:1019800032DA394B1B88002B31D12021039B9B6815
:101990008B4303998B600421059B34481B690B40E2
:1019A000FAD18024089989682143089CA1604024C9
:1019B0008168A14381600220079989688143079863
:1019C000816026492648C978490001801F4801687E
:1019D0002143016019001278D2B2069218AA9952D6
:1019E0000233802BFAD102E01378DBB20693204B4E
:1019F0001A88002A00D18AE200221A80029A1D4B1E
:101A0000126BD20700D482E21A6B104C3A431A636D
:101A10002168194AC90331D41968890304D511789A
:101A200018684B0018A9C852029B5B689B0329D514
:101A30001049137849685B0058A8C15222E0C0469B
:101A4000E60200203C0500203B0400207C0700202B
:101A5000FFFFFFFB7205002068050020E702002061
:101A6000A0020020DC020020E0020020C040005064
:101A70003E05002000000E402203002023680E993E
:101A80000B402360029BDB699B0309D5137838A8C0
:101A9000DBB2591CC9B21170CD495B00C969C15292
:101AA0003F2311780B401370FA22029B12011B682E
:101AB0009BB2934200D8DAE0C64B1B785BB2002B96
:101AC00000DBD4E0202240202368C3491343236075
:101AD0008A78C24B1A80226802420BD02268824365
:101AE0002260CA78198852008A1892B21A8000229D
:101AF000BB4B1A8080214020BA4B9A688A439A6077
:101B0000B94A9168014391603C381569B64905426C
:101B1000FBD1802598682843986040208B688343D8
:101B20008B60B24B1B88002BFBD000210720AF4BF2
:101B30001980AF490B68834380203B430B60029BB5
:101B400000011B6A0343029803620298A04B006BDA
:101B5000C007FAD50025186B38431863A5480570EF
:101B60001868A54D80B2A84204D99C4B1B88002B55
:101B7000C0D12BE007260868B043802638430860B0
:101B8000186A3601304318620298914B006BC00707
:101B9000FAD5186B38431863186880B2A842E4D8A5
:101BA00007260868B043384308608020196A00019E
:101BB00001431962186B8649C007FBD50B6B3B4389
:101BC0000B630B689BB2AB42CFD850E0FA21029B6B
:101BD00009011B689BB28B4249D98021814B874800
:101BE0009B688B437F498B60402193680B439360D4
:101BF00003228021824BC9031A70764B814A1F70E1
:101C000013680B43804913600B780133DBB20B7010
:101C10007E4B18800D78704B7D48052D0AD99D7A32
:101C2000002D01D09B7A00E05B7ADBB203700023C9
:101C30000B7002E05B7ADBB203700021754B1980F8
:101C40001168754B0B401360744B1A88002A0ED133
:101C50002021734A1A80734A93680B439360236868
:101C60005B0304D51422704B1F60704B1A60202256
:101C70000721236893435E4A236013688B433B43E9
:101C800013608022029B12011B6A1343029A1362A3
:101C900000231A00180018A9595A0D1C914200D2AD
:101CA000151CAAB29508A94201D2801800E040187C
:101CB0000233802BEFD13E2104F0B2FF464DC3B278
:101CC0000A932B7D984201D2287DC0B22B7D6421DE
:101CD000C01AAF235B00584304F0A2FF544B1A68AC
:101CE000801840081860FA232A799B005343414A20
:101CF000984201D20023137023685B0601D50023AC
:101D000013708023374E31690B4000D11370A978CE
:101D10001378994246D20023137080224021B36881
:101D20009343314AB36093680B439360032280214D
:101D3000334BC9031A70274B324A1F7013680B4389
:101D4000314913600B780133DBB20B702B4B9C468F
:101D500060462E4B18800B782D48052B04D9AB7AA2
:101D6000DBB20370002302E001006B7ADBB20B7080
:101D70000021284B19801168274B0B401360274B1B
:101D80001A88002A0ED12021254A1A80254A9368F4
:101D90000B43936023685B0304D51422224B1F601E
:101DA000224B1A60224B234A1B680F2B4AD9CF2B98
:101DB00002D89B080C3345E01F498B4202D81B090F
:101DC00033333FE01D498B423AD89B096C3339E0ED
:101DD00000000E4072050020E70200208E07002060
:101DE000A002002000400050C04000503E050020EE
:101DF00030000E40490500209F0F000088130000AE
:101E0000AC020020680500204805002020030020C7
:101E100066050020AE020020FFFFFFBFBA020020CF
:101E2000DC05000080400050704200504405002056
:101E3000B801002011030020FF040000FF1400007F
:101E40001B0A553B00242000DBB2137038ABE35A69
:101E50000234C018802CF9D1CE4B80095843CE4BA8
:101E6000000B98422AD864235B425843CB4BAF21E6
:101E7000C01804F0D5FEC3B20493502B20D9B36828
:101E8000C748A343B360C74B403C9A6822439A605B
:101E9000022202709968214380249960C24BE400B9
:101EA000196821431960C1490A7000210270C04AB3
:101EB00011801968BF4A0A401A6016E00023049393
:101EC000B94B1A68520510D5049A402A0DD81A68E1
:101ED0000F990A401A600022B44B1A70B64B197859
:101EE000AF4B032900D106321A700022130058A804
:101EF00011007E31415A023A5B1811007E31F7D150
:101F0000FA229B09520053431B0BDBB20C93A648E9
:101F100003683B4201D1FFF783FA0F21A74B1A78E0
:101F20008A43C02A0ED19A78D2B25A70DA78D2B2E5
:101F30009A701A79D2B2DA705A79D2B21A719A7941
:101F4000D2B25A710F215A788A43E02A00D01AE19E
:101F50005978D43A0A400C2A00D014E18025924ADC
:101F60005C7899781668ED05E4B2C9B22E4200D1CA
:101F7000F6E0DB783E2B09D00521894B1970002152
:101F80008B4B198011688B4B0B4013608B4AD378B5
:101F9000DBB2382B00D1A3E037D82C2B14D82A2B56
:101FA00078D2182B07D80A2B67D2082B00D0EAE08A
:101FB0003E21FF206BE0223B062B00D9E3E0D178E5
:101FC00008201E39C9B262E0352B6FD00DD8332BF3
:101FD00063D0342B00D0D6E0794C04206179B9432A
:101FE000FEF728FE6379BB4372E0362B72D0372BA5
:101FF00000D0C8E008260425714C042061793143E3
:10200000FEF718FE6179A9435AE06D2B1BD8642BAB
:1020100037D2492B71D0644A0CD8472B64D0482B57
:1020200000D0B0E01168674B654C0B4013606179DC
:1020300020257CE04B2B73D062D34C2B00D0A2E048
:10204000036880227AE0812B09D8782B00D380E0C6
:102050001423D17802206D395943C9B217E0FF2B00
:1020600000D090E00A991320FEF7E4FD6A4628218B
:102070005218534B12781A7585E0D1780020C9B2F6
:1020800005E00A230920D17864395943C9B2FEF723
:10209000D1FD78E0D17828395FE0494C042061799E
:1020A0003943FEF7C7FD63793B4311E00425082659
:1020B000434C280061792943FEF7BCFD6179B143A7
:1020C0002800FEF7B7FD63791D4365716379B3435B
:1020D000637158E004253A4C28006179A94328E04F
:1020E000374C0825617922E08021136849030B43AE
:1020F000334C1360617920250AE0036881221DE0DA
:1021000080211025136849040B432D4C136061791D
:1021100029430420FEF78EFD63791D43657132E08B
:1021200010251168284B264C0B4013606179042060
:10213000A943FEF77FFD6379AB43C9E7520513431B
:1021400009220360164B1A706A46194B928D1A8049
:1021500019E02823D17877395943C9B2032096E78B
:102160000320044024026418062C0CD1DB783E2B9B
:1021700009D169460E4B898D198013681D4315607E
:102180000822074B1A70084A1368BB431360FFF715
:1021900047F9C04688130000DE020000B81E0100A7
:1021A000AC020020C04000506805002072050020ED
:1021B000AE020020FFFFFFBF90070020FD020020BD
:1021C000E7020020FFFFEFFFFFFFFFFE07B5094A10
:1021D000136A0093084B196A019100991162019AE0
:1021E0001A62064B1B68002B02D000980199984791
:1021F00007BDC0460040005040400050DC010020B8
:102200001FB50C240D480E49036A0E4A01930B6A50
:102210000293136A0393029BA3430293019B0362FD
:10222000029B0B62039B1362074B5B68002B03D07E
:1022300001980299039A98471FBDC04680400050FC
:10224000C040005000410050DC0100200822044B37
:1022500010B51A62034B9B68002B00D0984710BD45
:10226000C0400050DC010020094B800182B0C01842
:1022700001900198019B1A6801238B402021134390
:1022800003600020034A13680B43136002B07047D9
:10229000144000508041005010B50F2811D80F2372
:1022A000094A184014689C430E3B19400B01102149
:1022B000204310601068884301001943116000201A
:1022C00000E0024810BDC046804100500189FFFF78
:1022D000F7B5264C0194002907D1019D019906000C
:1022E0000C6801211036B14012E0012904D1019D92
:1022F000019C814024680BE002290BD1019D0199CA
:1023000006000C6801210F001036B74081403943A8
:102310002143296016490191019C0121002A05D120
:102320008140019A12688A43226004E08140019A48
:10233000126811432160C0210E4A8900022808D189
:1023400050580D4B03408020000403435350042396
:1023500009E00A4883608020535800061B021B0ACC
:1023600003435350082300201360FEBDDC4000509F
:10237000D840005000E100E0FFFF00FFDC0100203A
:1023800030B5031E1D2B00D9C6E004F035FC0F1B31
:1023900022292B32323232323232323E444A5056C5
:1023A0005D6371808080808E8EA19ABC00205B4B23
:1023B00018605B4B18605B4B18605B4B18605B4BA5
:1023C0001860AAE0584A5A4B11680B408021C90195
:1023D0009EE0554A574B11680B40C021890197E098
:1023E0004F4A00E04D4A1168534B0B40F02109025F
:1023F0008EE001221500DC1CA540053B9A404848B0
:102400000168A9430A43026084E0474A4B4B1168C4
:102410000B4004217CE0444A494B11680B400821E1
:1024200076E0414A474B11680B40102170E03E4A6C
:10243000454B11680B4020216AE0394A434B116833
:102440000B408021490063E0354A414B11680B4045
:1024500080211AE0344A3F4B11680B4003210B43A3
:1024600013602E4A3C4B11680B40C02109014FE01C
:102470002B4A394B11680B40C02109010B431360F3
:10248000264A344B11680B40C021890040E0113BC3
:10249000590003230C001D00083C8B40A540214837
:1024A00002681343AB43036034E0204A11681928E3
:1024B00003D1284B0B4003212AE0274B0B400C2172
:1024C00026E0FF21174A13681B0C1B040B43136003
:1024D000FF21124A13681B0C1B040B431360124AA2
:1024E000174B11680B40802109010B4313601168E1
:1024F0001A4B0B40C0210B4313600C4A0D4B116863
:102500000B40302104E0094A144B11680B40C021F4
:102510000B431360002000E0114830BD3000005034
:1025200034000050380000503C0000504000005083
:10253000BFBFFFFFCFCFFFFF0F0FFFFFFBFBFFFF73
:10254000F7F7FFFFEFEFFFFFDFDFFFFFFEFEFFFF0D
:10255000FDFDFFFFFCFCFFFFF3F3FFFF3F3FFFFF2D
:102560000189FFFFF8B501232A4C25681D4205D0DB
:102570002360294B1B68002B00D0984702231D4283
:1025800005D02360244B9B68002B00D09847042380
:102590001D4205D02360204B1B69002B00D09847BB
:1025A00008231D4205D023601B4B9B69002B00D0E4
:1025B00098471A4D1A4C2F682668FB0608D52A68DA
:1025C000184B13402B60144B5B68002B00D09847CE
:1025D000FB0208D52A68144B13402B600E4BDB68B6
:1025E000002B00D09847F30608D522680D4B134006
:1025F0002360094B5B69002B00D09847F30208D594
:102600002268094B13402360034BDB69002B00D089
:102610009847F8BD44000440E80100205000044001
:10262000540004401F000F000F001F00F8B50123E5
:102630002A4C25681D4205D02360294B1B6A002BBC
:1026400000D0984702231D4205D02360244B9B6A8B
:10265000002B00D0984704231D4205D02360204B57
:102660001B6B002B00D0984708231D4205D0236028
:102670001B4B9B6B002B00D098471A4D1A4C2F68B0
:102680002668FB0608D52A68184B13402B60144BAC
:102690005B6A002B00D09847FB0208D52A68144BD0
:1026A00013402B600E4BDB6A002B00D09847F306DB
:1026B00008D522680D4B13402360094B5B6B002B40
:1026C00000D09847F30208D52268094B13402360D5
:1026D000034BDB6B002B00D09847F8BD440014403F
:1026E000E801002050001440540014401F000F0067
:1026F0000F001F00F021084A090413680B43C02192
:102700001360064B89031A680A431A601968044A61
:102710000A401A607047C046080200500C00005082
:10272000FFFFCFFF07230340043BDAB230B5032A93
:102730000ED93824C5002540373CAC4000251E4A40
:102740001368A343A94200D025002B4313600CE07B
:1027500001251A4CDB0022689D4013000022AB4388
:10276000914200D02A0013432360C30622D51038BB
:1027700007281FD804F040FA0406080A0C0E1016A9
:102780000F4A0AE00E4A0EE00E4A06E00D4A0AE041
:102790000D4A02E00C4A06E00C4A11680C4B0B4053
:1027A000082105E0094A11680A4B0B408021090302
:1027B0000B43136030BDC0460800044008001440BD
:1027C0005000044054000440500014405400144091
:1027D00007000F000F00070007230200F0B51A40A2
:1027E00085B00192023A00900D00AC4B052A05D845
:1027F000100004F001FA060608080B0B5B699B0049
:1028000006E05B6904E0DB699B0601E0DB691B060F
:102810009B0F04D0022B04D1A14B1B6802E0A14BFB
:1028200000E0A14B0293009B172B40D8180004F046
:10283000E3F90C0C0C0C121212123E3E3E3E3E3ED0
:102840003E3E222426282A2C2E36009B9748DC0068
:102850000168023404E09648009B0168DC001E3CDD
:102860000123A3400024EE689943A64200D01C0037
:1028700023000B431AE08F490AE08E4810E08E498E
:1028800006E08D480CE08D4902E08C4808E08C4958
:1028900008688C4B0340E86803430B6007E08848F6
:1028A000E96803680C0487490B4023430360019BDC
:1028B0002E781F1FFBB2032B11D900997B48CC0047
:1028C00038212140012403318C4003682100A343B7
:1028D0000024A64200D00C00234303600CE001203A
:1028E000FC000334A040002471490B688343A642D6
:1028F00000D0040023430B606968002966D1EB789F
:10290000052A05D8100004F077F9050507070C0C17
:102910006D4902E06C4905E06C49FF200A6882437A
:1029200004E06A4908681A02694B034013430B60CC
:102930006878AC686421604304F072F9AA78FBB24D
:1029400001380392032B18D9009A624B91001C2284
:102950001140153A17008F401E68BE43039F174071
:102960003A008A4016431E600C23019A611E5343AD
:10297000594A9A181160594A14E0594BBA0019681B
:1029800007231E009640B143039E1E403300934030
:102990001943534B534A19600C237B43611E9A1809
:1029A0001160514A9B181860AB780126032B01D89F
:1029B0004E4AD65CE9780298013104F031F93100D1
:1029C00004F02EF9210004F02BF9F9E0029804F04C
:1029D00027F9802307005B0500209F4200D9EFE024
:1029E000434B9F422ED9390C38008CB204F018F9B1
:1029F00080235B02984201D90134A4B280235B009A
:102A00009C4220D93C0A390E2000CEB204F008F9CD
:102A100080235B02984201D90136F6B200230120DF
:102A20000200591C9A40CBB2B242F9DD0126013BAB
:102A30009E40F6B20020102E00D9C1E0270280246B
:102A4000640001E0022401262100380004F0E8F8C7
:102A5000310004F0E5F8070083B2210002980393E7
:102A600004F0DEF8310004F0DBF8B9B204F0D8F875
:102A7000019B0290981E013C052804D804F0BCF884
:102A8000050507073A3A104A02E00F4A33E00F4AB9
:102A9000FF2113680C408B4332E0C0460002005017
:102AA000F8000020001BB70000805101080004401E
:102AB00008001440500004405400044050001440EA
:102AC000540014400F000F000000044000001440A8
:102AD000FF00FFFF040004400C000440100004400D
:102AE000040014400C00144010001440406F00001B
:102AF000FFFF0100334AE4B211682302324C0C405C
:102B00001C43701E14600F2812D804F075F81008CA
:102B1000110A1111110C111111111111110E0026B0
:102B200006E0012604E0022602E0032600E0042677
:102B3000009B6878DB0607D5AB6864215F1E5843AD
:102B4000BFB204F06DF807E0039B013F43436421EB
:102B50001800BFB204F0EEF8019B01381A1FD3B27F
:102B600080B2032B17D9009B184C99001C231940E5
:102B7000153B1D001E408D408E4022680533AA4340
:102B800032432260019A5343114A9A181760114A3E
:102B90009B18186013E007219500A9400E4C23688C
:102BA0008B43190007231E40AE4005335A430B4B9D
:102BB0003143D31821601F60094BD218106002986E
:102BC00005B0F0BD00001440FF00FFFF040004400A
:102BD0000C00044010000440040014400C00144099
:102BE000100014401023042200291CD018420ED0DB
:102BF000104204D01C4914388A6F0F3B04E00723AD
:102C00001A4918408A6F063B834013431BE0012397
:102C1000104203D0164904380A6801E015490A68D1
:102C2000834013431DE018420FD0104204D00E49D8
:102C300014388B6F033A04E007220C4910408B6F65
:102C4000063A824093438B670CE00123104203D085
:102C5000074904380A6801E006490A6883409A4334
:102C600013000B607047C046000014400000044091
:102C70007C0014407C00044007221040023800B55C
:102C80000323124A052804D803F0B6FF09091111DD
:102C900016160B40506919070D4B034004E05069AC
:102CA0000B40990783009B080B4353610CE00B40DA
:102CB0001901D069302303E00B409901C023D0698A
:102CC000984303000B43D36100BDC046000200508F
:102CD000FFFFFFCF0022044B5A60586801231840C1
:102CE000904200D001487047FC0000500296FFFF60
:102CF000A0220121D20593680B4393607047000026
:102D0000A022102110B5D20593690B439361034BA8
:102D10001B68002B00D0984710BDC0462802002039
:102D200010B50123232805D10E480B40D900426875
:102D3000082306E0222809D10B4099000423094802
:102D400042689A4313000B43436009E0064C8340FA
:102D50002268002902D01343236001E09A432260D5
:102D600010BDC0460002005008020050402110B5BE
:102D7000044A13680B431360034B5B68002B00D0BD
:102D8000984710BD000200502802002000487047FC
:102D9000001BB70030B585B06A46134B6D4613CBA8
:102DA00013C21B681360114B1A6A120301D4104A34
:102DB00000E0104A1B6A0D4C0020DB0311D4206A8E
:102DC000216A246AC005C00D89042404C90EA40F19
:102DD000023002315043A40003F022FF295903F0CE
:102DE0001FFF05B030BDC046446F00000002005018
:102DF000001BB7000080510110B50E4C23695B0722
:102E00000ED023695B075B0F022B02D1FFF7C2FFD5
:102E100009E023695B075B0F032B03D0064802E040
:102E2000064800E00648A1690907090F013103F0CF
:102E3000F7FE10BD0002005000805101001BB700DA
:102E400010270000F7B504218020D24BD24ADC685D
:102E500011621968C0040143802019601968C00517
:102E6000014319600021CD4BCD48198003680092C1
:102E70009B063AD4CB4B1D781900092D35D8CA4D85
:102E80002E68B2000FD4C94E3678002E0BD02968B8
:102E90004A052AD429684A0227D419780131C9B2CF
:102EA00019701B7809E0C24B1B78DBB2002B17D0DE
:102EB0000B780133DBB20B700B780A2B15D1802510
:102EC0000521BC4B1D70BC4B1970BC498B682B4352
:102ED0008B604021009B009A9B688B43936004E0C9
:102EE0000725B5490D70B3490B700021B44B19800B
:102EF000642C00D8BDE10225AB490E680B002E42C0
:102F000000D18BE10E680E352E4202D00B68AB4328
:102F100014E00E68AB4DB20600D41CE104260F6825
:102F200037420DD140200B681E430E600A68824371
:102F30000A60AC4200D99CE10B6803430B6098E146
:102F400080270968B14319601E68BE431E60AC4209
:102F500002D81968394319601C689B49220600D4BD
:102F6000E5E00427994CA5687D40A5600D78012D0A
:102F700000D875E10126964DB4466D79354237D0BB
:102F8000944D2E6A3200944E164062462E62934E45
:102F9000F76780272E6AFF0596432E62904E3568AC
:102FA0003D430027356008268E4D2F70A5683543B8
:102FB000A56040258026009A760294682C43946090
:102FC0000568894C354305602770884C2578FF2DAE
:102FD0000FD165780324A543FC2D0AD1844DAC683C
:102FE0003443AC60802504686D012C43046000E02C
:102FF0000878804E0C7835787C48E4B2EDB20555FF
:103000000024250001960E78B44204D8065D0134F0
:103010007540E4B2F7E7002D00D021E13F260478A7
:10302000B443802C5FD11968CA000CD50178724C6A
:10303000C9B221704178714CC9B2217080241968DD
:10304000A4002143196062494C79E2060FD5CD7A7C
:103050000478A5420BD10D7B4478A54207D1802589
:103060001C686D042C4300251C60654C25804C7940
:10307000A20600D4F4E04D7B0478A54200D0EFE036
:1030800001248D7B4178A143A94200D0E8E041783A
:10309000484E2140484D0BD00021424A11708022F9
:1030A00032701968574A0A401A6005222A70D7E020
:1030B00002225548876817438760876892189743AC
:1030C00087603E4F7C32B8689043B8604027009AD2
:1030D000906838439060317081211A6889050A43ED
:1030E0001A602C70BCE01A68484C494E22431A60A2
:1030F0002A00484C257000940C783700A446541CD4
:10310000E4B2944505D9855CEDB2B55401252200A1
:10311000F2E7002D01D00098027001980A7800783B
:10312000D2B2C0B2B854F2201A6882431A60314851
:103130000A7800782D4CD2B2C0B2A05420201A6870
:1031400082431A600A780132D2B20A700A78102AD1
:1031500000D985E08DE027490A785200D2B20A7082
:10316000AC4203D80A780132D2B20A702A490A78EE
:103170000132D2B20A700A78072A05D920201A68CB
:1031800002431A6000220A7010211A680A431A606A
:103190006FE0C04620001140C04000506C05002088
:1031A0007C0700206E050020680500201203002027
:1031B0006205002072050020AC0200200040005093
:1031C00070050020FF0700003A04002080400050F6
:1031D000E702002000000E40FFF7FFFF04E100E0DF
:1031E00000001140B80200203B050020BC02002076
:1031F0000002005013030020230300207807002062
:1032000082070020FFFFBFDF0041005001000800DF
:10321000FD02002030020020750700201549164AE3
:103220008C4219D9117812291AD91968490702D57F
:103230001968294319600420196801431960196845
:10324000890716D51968FB30814319601968F5386C
:1032500001431960002309E013780133DBB207E072
:103260001968064A0A401A600023034A1370044A88
:103270001370F7BDFF0700007507002000FFFEFF79
:103280003A04002008222F4B2F49F0B51A620A6831
:103290002E4B13402E4A0B6013685B0350D58024DD
:1032A0001068A4022B4B204206D110682043106006
:1032B00080201C78204306E01468274820401060D6
:1032C0007F201C7820401870802005250B68C004E2
:1032D00003430B60214B224F1C78E4B2601CC0B248
:1032E0001870204805551C78E4B2651CEDB21D70BD
:1032F000042505551C78E4B2651CEDB21D7000254F
:1033000005551C78E4B2651CEDB21D703D78EDB238
:103310006E1CF6B23E7005551C78E4B2651CEDB229
:103320001D70872505551C78E4B2651CEDB21D7033
:1033300013689B03DB0F03550A680B4B13400B60AC
:10334000F0BDC046C040005068050020FFFFDFFF11
:103350007C070020AC020020FFFFFDFFE6020020FA
:103360003C0500203B040020FFFFFFFBF7B5C64AE9
:10337000C64C1388019401339BB21380C44A13884E
:1033800001339BB213802388002B03D02388013B99
:103390009BB22380BF4A13780133DBB21370BE4B5C
:1033A0001A68002A02D01A68013A1A60BB4A1388C8
:1033B000002B06D1BA4BBB481A68BB4ED2010FD4C2
:1033C00041E01388013B9BB2138013889BB2002B12
:1033D000F0D11900B54AD15401330A2BFBD1E9E7EA
:1033E000B34AB4491278802A03D10A88013292B2D2
:1033F00000E000220A800988AF4A914223D9802543
:10340000AE4981278A689024AA438A60AC49403D2E
:103410008A68BF052A438A600021AA4A3C3D15708C
:10342000A34A11701A683A431A600768A64A3A40DC
:10343000A64F0260BA682243BA608027A44ABF013F
:10344000D767D5673170A3490A88002A0BD00A884C
:1034500092B2551EADB20D80012A04D120259B49A0
:103460008A68AA438A609C490A88013292B20A801B
:103470009A490A88002A03D00A88013A92B20A803F
:10348000974D984A298800290CD02988013989B29A
:103490002980954911802988002903D14025016898
:1034A000A94301601188002909D01188013989B226
:1034B0001180128892B2002A01D18C490A708C497D
:1034C0000A78D2B2002A0ED0FA278A4DBF006A8845
:1034D000BA4202D801326A8014E000226A800A7877
:1034E000013AD2B20DE08449097800290AD0704926
:1034F000097849B2002905DB1D6880492940196017
:103500007F490A707F4A118889B24D1CADB215807F
:10351000C8291DD18027694DA968B943A960684DA4
:10352000403FA9683943A9600021754D3A3F297091
:10353000754D29801D687549294019605C49614DA8
:103540000F703178C9B2002901D1297000E02F70C5
:103550001288C72A21D81A6852041ED50021402794
:10356000674A564D1170AA6880310A43AA60544DCB
:10357000AA68BA43AA604E4A1170524A7B39117048
:103580001968634A0A4080211A600268C9040A4324
:10359000026019685F4A0A401A605F4A1168002990
:1035A00007D01168013911601268002A01D15B4906
:1035B0000A605B498A79002A0FD04E4A97887D1CA1
:1035C00095800A258C796543AF4206D180271D6816
:1035D0003F043D431D6000259580524A1588013502
:1035E000ADB215803578EDB2002D00D1AEE04E4D74
:1035F000296801312960C8212F6889008F4200D8CD
:10360000C5E000212960494D2F680F253D40484FF6
:1036100040353D709027474D31702970464D2B4EF7
:103620002970B5683D43B5600126334D103F2E70BB
:10363000224EB568BD43B560214E403FB5683D435D
:10364000B560204D019C29702F4D29801E682F4D9B
:10365000354004261D60394D2E60FA25AD002580C9
:103660000625134C2570264C21701D68284C2540DA
:103670001D60334C02252170324C217032498C6818
:1036800034438C608C6879E024030020E002002041
:103690007607002049050020DC02002036030020C8
:1036A000680500207C0700209007002014030020FC
:1036B0007205002082070020B03600000040005054
:1036C000C0400050AC020020FFFFFBFF80400050D4
:1036D00004E100E0BA0200203E0500208E07002031
:1036E000A0020020200300208813000048050020CD
:1036F000660500203002002012030020FFFFBFFFFC
:103700006E05002070050020AE020020FFFFFFBF05
:10371000FFFFBFDFFFBFFFFF4405002070420050E6
:10372000E70200206405002088070020B402002082
:1037300039040020740700209107002000E100E018
:10374000E60200208407002000001540497949075F
:103750001DD5874C218889B24E1CB6B22680FA2628
:10376000B600B14213D92580102582490C692C423C
:1037700006D08C68AC438C608C6870352C4305E0B7
:103780008C682C4380258C608C68AC438C608021D5
:1037900000688902084035D01388DBB2802B00D046
:1037A000E5E0754A754B9179012916D000290AD0B8
:1037B00002291ED1986801430420996099688143C9
:1037C0009960032313E00420996801439960996884
:1037D000023881439960012309E00220042499689A
:1037E000014399609968214399609071BFE093719A
:1037F000BDE0002191719A6802318A439A609A680B
:103800000231B2E05E495F4C0D88002D13D00D8867
:10381000012D0CD11E685C4D35401D605B4B1B7843
:103820005BB2002B02DA0523237000E020700B88C6
:10383000013B9BB20B802078C0B2092800D996E0EA
:1038400003F0DAF905132A303D5C61777B82FA22B6
:103850004F4B92001988914200D088E00022042149
:103860001A80464A93684B403FE013888022DB056C
:10387000DB0D5200934200D079E03F4BD879421CD7
:10388000DA71052873D803F0B7F9033203327236C0
:103890003A4A0421936827E012880221374B9206A6
:1038A0000BD504E012880221344B120605D59A6824
:1038B0000A439A609A68491857E09A6855E0138855
:1038C0008022DB05DB0D5200934250D12A4BD87980
:1038D000421CDA7105284AD803F08EF9030903095E
:1038E000490D0221254A93680B4393603FE0234B27
:1038F00004219A6835E00022DA7138E004211F4B78
:103900009A680A432EE0FA22214B920019889142CC
:103910002DD100221A80184B1A7A511C19720421D9
:10392000164BD2071CD49A680A439A609A680221FF
:1039300014E0124B04219A680CE0128804210F4B0A
:1039400052060DD59A6809E0128804210B4B5206E5
:1039500006D59A680A439A609A6802390A4305E0D4
:103960009A688A4302219A609A688A439A60F7BDEE
:103970006C050020804000503002002000410050C3
:10398000AE020020AC020020FFFFFFBF7205002046
:10399000700500208021DF4AF0B5136849020B430F
:1039A000DD491360087885B0C0B2431CDBB20B70F0
:1039B000042801D900F0A0FD8023DB0503F01CF9E9
:1039C000080E080328000820D4498A6882438A60C8
:1039D000D3490A6813430B6000F08EFDD04801689C
:1039E0000B4303600820CD498B6883438B601368C9
:1039F0005B0305D58021CB4A490293680B43936052
:103A00000221C94B9A680A439A601B6800F074FD52
:103A10008020C649C0040B78013BDBB20B70C44B5D
:103A200019680143802019601968C00501431960B5
:103A3000C049D8688842FCD900210124BE4B1970C6
:103A4000BE4B1970BE4B186A2043B64C1862A5686D
:103A5000BC482840A0604024BB4DA868A043A86093
:103A60000425BA4805608025186A2D01284318628C
:103A7000B7484379234201D100F0ACFCB54B1C7828
:103A80001D008C4201D100F0A5FC1C780F2C01D840
:103A900000F0A0FC1C78EF2C01D900F09BFC1B78F7
:103AA000AD4E0F3BDBB2F35CDBB2402B25D113688C
:103AB000DB0401D400F08EFC13685B0301D400F03A
:103AC00089FC80220A25A548D204036813430360B9
:103AD000A34B1C78E4B2621CD2B21A70A14A1555ED
:103AE0001C78E4B2651CEDB21D70092515551C78D3
:103AF000E4B2651CEDB21D7034E29C08E7B2072FFA
:103B000044D003D8002F07D000F064FC0E3C012CF9
:103B100000D8AAE100F05EFC69780E2901D800F017
:103B200059FC002490490C6069780F39715CC9B266
:103B30000291402901D100F04DFC8C49087840B237
:103B4000A04203DA3F200C78044008E08878C0B235
:103B5000C8704878C0B288700878C0B248700194C4
:103B60000F248878A0430024E02801D08C70CC700A
:103B700000207F4C275C0E5C2500B74201D000F08E
:103B800040FC01300528F5D100F045FC6C780E2C86
:103B900001D800F01FFC744C2160A9780F2907D9C7
:103BA000E978EF2904D8AB780F3BDBB2F35CDBB2EA
:103BB000012B06D0002B06D0072B00D195E000F09A
:103BC00009FC80235B0029780F39C9B2775C6978DA
:103BD000FFB20F39C9B2755C6449EDB20C7864B2BA
:103BE000002C01DA0C7808E08C78E4B2CC704C78C8
:103BF000E4B28C700C78E4B24C7000240E7801941E
:103C000076B2A64203DA0C783F210C400194126888
:103C1000520300D4DEE3BA01AA18564DD2B2698924
:103C200052189B189BB25B086B81427952B2002AF2
:103C300000DBCFE30A2250490D88C07C4243954205
:103C400000DCC7E300260E80802108274348C90412
:103C500002680A430260424A1578EDB2691CC9B293
:103C6000117040494F551578EDB26F1CFFB21770B7
:103C700007274F551578EDB26F1CFFB217704E55E0
:103C80001578EDB26E1CF6B216703C4EB446644622
:103C90003678F6B2771CFFB227704E5515786C4611
:103CA000EDB26E1CF6B21670A6264E551578247924
:103CB000EDB26E1CF6B216702C4E7678F6B24E55FA
:103CC0001578EDB26E1CF6B216704C551478E4B24D
:103CD000651CEDB21570DDB20D5514781B0AE4B207
:103CE000651CEDB215700B5575E12B780F3BDBB2FF
:103CF000F15CCBB201936B780F3BDBB2F35CDBB2D0
:103D000002931A4B1C7864B2002C39DA1C783F23DA
:103D10001C403FE07C070020B8020020804000509B
:103D20000000114000020050000005402203002066
:103D30002000114061020000750700203A040020B5
:103D400000000E40FFFFFEFFC040005000E100E019
:103D5000E7020020A20200200000002068050020E9
:103D6000E60200203B04002070420050BC0200200C
:103D70001403002030020020240300203C05002012
:103D80009C78E4B2DC705C78E4B29C701C78E4B29D
:103D90005C700024837C002B00D11BE36423EC4D7A
:103DA0002E88807C43439E4200DC13E300262E8055
:103DB00013685B0300D40DE380220927E548D20491
:103DC000036813430360E44B1D78EDB26A1CD2B262
:103DD0001A70E24A57551D78EDB26F1CFFB21F7082
:103DE000082757551D78EDB26F1CFFB21F7056554E
:103DF0001D78EDB26E1CF6B21E70D94EB446614607
:103E00003678F6B2771CFFB20F7056551D78EDB2BA
:103E10006E1CF6B21E70AA2656551D78EDB26E1CA9
:103E2000F6B21E70FF2656551D78EDB26E1CF6B226
:103E30001E70CC4E7678F6B256551D78EDB26E1CDB
:103E4000F6B21E7054551C78E4B2651CEDB21D70BC
:103E5000012515551C78E4B26519EDB21D70019B62
:103E60009901029B5918C9B2B4E01168C90400D481
:103E7000B0E20020BC499B010860DCB26B78B94914
:103E80000F3BF35C4878DBB2FB38042800D9A1E291
:103E900002F0BCFEFC0105000500A600A600802182
:103EA000C902402B3ED012680A4200D192E2802122
:103EB0000A26A84AC90412680A43A6490A60A64A03
:103EC0001078C0B2411CC9B21170A4490E541078C8
:103ED000C0B2461CF6B2167009260E541078C0B255
:103EE000461CF6B2167000260E541078C0B2461C5E
:103EF000F6B216709A4EB44665463678F6B2771C1E
:103F0000FFB22F700E541078C0B2461CF6B2167075
:103F1000B3260E541078C0B2461CF6B21670FF26B7
:103F20000E54C9E013680B4200D153E280220A24E8
:103F30008848D204036813430360874B1978C9B2D9
:103F40004A1CD2B21A70854A54541978C9B24C1C12
:103F5000E4B21C70092454541C78E4B2611CC9B248
:103F60001970002111551D787D4FEDB26C1CE4B223
:103F70001C703C78E4B2661CF6B23E7054551C7856
:103F8000E4B2651CEDB21D70B32515551C78E4B282
:103F9000651CEDB21D70FF2515551C78E4B2651C3B
:103FA000EDB21D7011551C78E4B2651CEDB21D70A8
:103FB00011551C78E4B2651CEDB21D7011551C78CA
:103FC000E4B2651CEDB21D7011551C78E4B2651C9D
:103FD000EDB21D7011550268644B13400360F9E1A6
:103FE0008020C002402B00D1C6E01268024200D1FE
:103FF000F0E180210F26574AC90412680A43554947
:104000000A60554A1078C0B2411CC9B211705349B8
:104010000E541078C0B2461CF6B2167004260E5428
:104020001078C0B2461CF6B2167000260E541078F6
:10403000C0B2461CF6B21670494EB4466546367894
:10404000F6B2771CFFB22F700E541078C0B2461C27
:10405000F6B21670B4260E541078C0B2461CF6B2F2
:104060001670FF260E541678F6B2701CC0B210708F
:104070003C488778FFB28F551678F6B2771CFFB2AE
:104080001770C778FFB28F551678F6B2771CFFB25B
:1040900017700779FFB28F551678F6B2771CFFB20A
:1040A00017704779FFB28F551678F6B2771CFFB2BA
:1040B00017708079C0B2885510782343C0B2461C6F
:1040C000F6B216702A4E0B54B3782A4C0F3BE35CC1
:1040D000F0789B010F38205CDBB203431078C0B24C
:1040E000471CFFB217700B5433790F3BE05C7379B8
:1040F00080000F3BE35CC0B2DBB21F093843009085
:10410000684617781B01FFB27D1C05710579009880
:104110001570C855B079DBB20F38205CC0B2870883
:104120003B4300936B4617788001FFB27D1C1D71E5
:104130001D79009B1570CB55F3790F3BE35C184359
:104140001378C0B2DBB25C1CE4B21470C8543BE11B
:104150007607002068050020E60200203B040020CE
:104160003C050020BC02002070420050FFFFFFFB16
:10417000A2020020000000201368034200D129E1C0
:1041800080220F25DD4CD204236813432360DC4BCF
:104190001878C0B2421CD2B21A70DA4A1554187894
:1041A000C0B2451CEDB21D70042515541D78EDB24A
:1041B000681CC0B21870002050551D78EDB26E1CFE
:1041C000F6B21E70D04E0195B44665463678F6B20A
:1041D000771CFFB22F70019D56551D78EDB26E1CF5
:1041E000F6B21E70B42656551D78EDB26E1CF6B2AE
:1041F0001E70FF2656551D78EDB26E1CF6B21E706D
:104200008E78F6B256551D78EDB26E1CF6B21E7061
:10421000CE78F6B256551D78EDB26E1CF6B21E7011
:104220000E79F6B256551D78EDB26E1CF6B21E70C0
:104230004E79F6B256551D78EDB26E1CF6B21E7070
:104240008979C9B251551978C9B24D1CEDB21D70AA
:1042500050541978C9B24D1CEDB21D7050541978E4
:10426000C9B24D1CEDB21D7050541978C9B24D1C25
:10427000EDB21D7050541978C9B24D1CEDB21D70CD
:1042800050542268A14B13402360A3E0402B00D17F
:10429000A0E01268520300D49CE080210A26974ACD
:1042A000C904126823430A4394490A60944A157862
:1042B000EDB2691CC9B2117092494E551578EDB234
:1042C0006E1CF6B2167009264E551578EDB26E1CAE
:1042D000F6B2167000264E551578EDB26E1CF6B289
:1042E0001670894EB44660463678F6B2771CFFB237
:1042F00007704E551578EDB26E1CF6B21670B526E5
:104300004E551578EDB26E1CF6B21670FF264E555E
:104310001578EDB26E1CF6B216707D4E4B55B37823
:104320007C4D0F3BEB5CF4789B010F3C2C5DDBB2CA
:1043300023431478E4B2671CFFB217700B5533792E
:104340000F3BEC5C7379A4000F3BEB5CE4B2DBB297
:104350001F093C4300946C4617781B01FFB2781C80
:1043600020712079DBB210700098C855B4790F3CE9
:104370002C5DE4B2A7083B4300936B461778A40179
:10438000FFB2781C18711879009B1070CB55F37927
:104390000F3BEB5C1C431378E4B2DBB25D1CEDB267
:1043A0001570CC5413785C4DDBB25C1CE4B2147015
:1043B000EC79E4B2CC541478E4B2631CDBB2137031
:1043C000C0232A7A13430B554C4B1A684F4B1340AA
:1043D0004A4A13601021514B1A680A4205D0032043
:1043E0004F4A10601A688A431A6019684D4A0A4099
:1043F0001A6000231900464AD1540133082BFBD11F
:104400007AE00023484A1373CA5CD2B2EA540133FB
:10441000052BF9D1DEE7444C207B451C2573012890
:10442000D8D11268520362D580200926334CC004CB
:1044300022689B0102432260314ADBB21578EDB25B
:10444000681CC0B210702F4846551578EDB26E1C2E
:10445000F6B21670082646551578EDB26E1CF6B207
:104460001670002646551578EDB26E1CF6B2167021
:10447000254E0395B44665463678F6B2771CFFB2F2
:104480002F70039D46551578EDB26E1CF6B216706E
:10449000A52646551578EDB26E1CF6B216704E780C
:1044A000F6B246551578EDB26E1CF6B216706E4631
:1044B000367946551578EDB26E1CF6B21670CE7888
:1044C000F6B246551578EDB26E1CF6B216708E78BF
:1044D0000321314041551178C9B24D1CEDB2157020
:1044E000029A134343542268084B13402360C822A6
:1044F0000E4B92001A806DE705B0F0BD68050020F4
:10450000E60200203B0400203C050020FFFFFFFBEB
:10451000A202002000000020BC0200207C07002036
:1045200044050020FFEFFFFF30020020360300208B
:10453000F7B56A46234BD01D1B680127DBB2037019
:1045400000231D001E001C0001781F4AC9B25173D0
:104550009373D373082B09D0394202D0012601345A
:10456000E4B201334908DBB20125F3E7002E00D0A5
:104570009473002D02D008235173D373937B042BC3
:104580001ED1124B1A68520306D50121104A116040
:104590001A680F310A431A600E490B78DBB25A1CB5
:1045A000D2B20A7002780C48D2B2C2540B78092BEE
:1045B00006D90023094A0B709168094B0B409360A0
:1045C000F7BDC04600000540300200207C070020F7
:1045D000704200503B050020A20200200002005063
:1045E000FFFFFEFFF0B5BA4C87B0236804AADBB228
:1045F000D11D0B70A3691B07DD0F002B00DB4AE107
:10460000082640277F22A3693343A36108780B78EB
:1046100038401340002800D1BCE07D2B00D1B5E02C
:104620007E2B00D0B4E2AB4D2B78002B00D08DE078
:104630008021A94A93688B439360A84A93681F43DB
:10464000A74B97601B78DBB2002B06D08021A54AD0
:10465000C90113680B43136004E00621A24A1170DC
:10466000A24A1370A24A1378DBB2002B03D013784E
:10467000013BDBB268E00B229E4D9F492A70013A54
:104680006A70E632AB70EB702A71EE3A6A713C32B6
:10469000AB71EA710A68120E2A720A68120CD2B261
:1046A0006A720A68120AD2B2AA720A680C21D2B2DD
:1046B000EA72924A1170924A1370924A1374894AAC
:1046C000914B11680B4013601022E3681343E360C1
:1046D000E36892181343E360E368183A1343E36016
:1046E000A369DB00FCD52E78794BF6B21E60300052
:1046F00000F016FB0127B74215D8A3691B02FCD4B2
:104700007F4A7349137801370133DBB21370EB5CD6
:10471000FFB2DBB20B601378DBB2EB5C5840C0B287
:1047200000F0FEFAE7E7A3691B02DB0FFBD1684A42
:10473000734910600A780132D2B20A70734A13705A
:10474000734A1360634A0233137040E22B78022BE2
:1047500000D03CE200F0D6FA0021654B6C4A18709C
:104760006C482970116011684C1C14608142FAD9A0
:10477000002111601A788A4200D028E25E4A12684D
:10478000D2B21A700F2219780A405BE00022604B07
:104790001A601CE2002B17D180245C486400027868
:1047A000D2B2511CC9B201705B4952005452027816
:1047B0005200535280210378524ADBB21374574A95
:1047C000090613680B435FE0424B1B78DBB2022BF8
:1047D0005CD0032B00D0DBE1514B09781A781F2302
:1047E0000B40934200D0F2E11021494A1060E36887
:1047F0000B43E360E36849180B43E360E36833432A
:10480000E3600292A3693249DB00FBD5354B1A689D
:104810008023DB041A4002D001230B60D7E1384B20
:1048200036481F7805781E00AF4201D10A60CEE1FC
:104830001A78304DD2B2AD5CEDB22A1F3B2A03D9B3
:104840000278D2B21A70C2E10D60280000F068FA56
:1048500001273378274A0133DBB23370D35C013749
:10486000DBB223603378FFB2DBB2D35C5840C0B216
:1048700000F056FABD42ECD2154B18603378029A1C
:104880000133DBB2337000231360A0E11D4B1D74B4
:104890001F4B18607CE1214A1C4D10681E4B0028FC
:1048A00000DB60E1174E307C40001F5AC0203840CA
:1048B000029037D011684900490811600021327C0C
:1048C000013AD2B22A702A78520099527FE1C0464A
:1048D000000015409007002000400050C0400050EC
:1048E0001203002068050020AC02002072050020A1
:1048F000390400203B040020B4020020E60200201E
:104900008C07002030020020FFFFFFFB84070020FF
:1049100088070020FFFF0F00740500207C0700209F
:10492000380400202F78F8B2019002AF0130F871FE
:10493000F8792870019809784700D953317C4900EB
:10494000595A002900D123E1317C49005F5A317C5A
:104950002E780231C919C9B2B14200D018E12978C4
:1049600002A8C9B24E1CF6B22E7080264900B600CD
:104970005E52297800884900585202981368060050
:104980005B005B081360934F934A3B7C39005B00EC
:104990009B5A0133B3420FDB3B7CF318DBB25B0065
:1049A0009B5A8E4ADBB29355935D01365840C0B294
:1049B00000F0B6F9F6B2E6E7894A1378DBB2022BCB
:1049C00005D0032B00D0E3E00022864BC9E0834BE7
:1049D000002804D000231370FF22834B32E71A799A
:1049E0001E00702A7ED100217E4F804E3960587A99
:1049F0003268120E904200D0CAE09A7AFF209446A4
:104A00003268120C0240944500D0C1E0DA7A944634
:104A10003268120A0240944500D0B9E01A7B366829
:104A20000640B24200D0B3E003226D4E32705B7993
:104A30006F4ADBB213701378DBB28B4203D1337051
:104A4000694B1870C3E039602B786A4ADBB2137087
:104A5000694B6A4A186802401A60694A6948557980
:104A6000AD0718D58027684E0170B568BD43B560A5
:104A7000664E403FB5683D43B560654D2970654958
:104A80000D78052D01D1023500E006250D700025B9
:104A900061490D7001E001210170102551799026C6
:104AA000A943517152790C3D5C492A4216D08A685B
:104AB000B2438A600278002A6AD00021584A1180E5
:104AC0001868584A02401A60574A1560524A1170D5
:104AD000564A11701968564A0A4042E08B683343BF
:104AE0008B6055E01A79722A1FD100253D4A3F4854
:104AF0001560597A0268120E914249D1FF219E7ABF
:104B00000268120C0A40964242D1DE7A0268120A0A
:104B10000A4096423CD11A7B03680B409A4237D137
:104B20002F4B1D70304B197051E018781F785A7850
:104B3000C0B2013297422BDD5A780132D2B20A74E8
:104B40000F7C1A78D21BD2B21A7000220132D7B26F
:104B5000B84200D843E70F7CBF18F75DFFB2B754E7
:104B6000F4E71A6014E02878013840001E5A8020CB
:104B7000400086420CD12878C0B2461CF6B22E7096
:104B80000978400019528021136809060B4313600D
:104B9000A369284A1B0403D5022193680B43936041
:104BA000A269244BD20707D501219A690A439A6169
:104BB0009A6849180A439A60A3699B0603D41D4B5F
:104BC0009B69DB0603D50222A3681343A36007B0E9
:104BD000F0BDC046300200207405002038030020DC
:104BE000900700208807002039040020B40200202C
:104BF000380400209107002068050020FFFFFBFF1C
:104C0000E70200201203002000400050C040005086
:104C100062050020AC020020720500208040005098
:104C2000AE020020FFFFFFBF00E100E06E050020A4
:104C3000FFFFBFDF0000154010B5FBF7EDFFFEF7EB
:104C400057F810BD70B51B4C1B4D23695B075B0FFC
:104C5000052B02D8022B04D000E004239B00E85867
:104C600019E00123266A3604B60FB3429B415B422A
:104C7000F61A236A1B0301D4104B00E0104B206A84
:104C8000216AC005C00D8904C90E023058430231A3
:104C900001F0C6FFF040A1690907090F013101F0D9
:104CA000BFFF084B68610849C01801F0B9FFA8614F
:104CB00070BDC04600020050E4000020001BB70099
:104CC0000080510120A1070040420F007047000002
:104CD0000B4B1A7819785200D2B24A405200197818
:104CE000D2B24A4012011978D2B24A401978D20998
:104CF00049005218D2B21A701878C0B27047C04634
:104D00004005002010B5FFF7E3FF0F23034A1840CA
:104D10001378C0181F231840107010BDB002002077
:104D20000023C20700D55E33820701D5BC22534061
:104D3000420701D561225340020701D5C2225340E8
:104D4000C20601D59D225340820601D5232253403D
:104D5000420601D54622534040B2002801DA8C2297
:104D60005340180070470000F0B5D24BD24C1A786F
:104D7000237893B09A4201D101F064FE8023227817
:104D8000CE4D5B00002A12D1FF32FF32AA5A190021
:104D90009A4202D18022520015E02378DBB25A1CDD
:104DA000D2B222705B00EB5A8B42F6D1F2E7227846
:104DB000013A5200AA5A9A42ECD02278D2B2511C3F
:104DC000C9B22170F5E723785B00EB5A934204D116
:104DD00023780133DBB22370F5E723785B00EB5ACD
:104DE000002B01D101F02EFE23785B00EB5A023339
:104DF000DBB20193019A2378D318DBB25B00EA5A45
:104E000080239B009A4201D001F01CFE0026300056
:104E10002378019AD318DBB25B00EE52019AF3B209
:104E20009A420FD92278D2B2531CDBB223705200BF
:104E3000AA5AD3B202AA93554340D8B2FFF770FFE3
:104E40000136EBE7802223789D490133DBB22370E2
:104E50000B68D20413430B60002845D0994B02AA7B
:104E60001B7892789A423FD100200625964B974FA7
:104E700018701C78E4B2621CD2B21A70944A1555AC
:104E80001C78E4B2651CEDB21D70052515551C7823
:104E9000E4B2651CEDB21D7010551C78E4B2651CBF
:104EA000EDB21D703D78EDB26E1CF6B23E70155538
:104EB0001C78E4B2651CEDB21D70862515551C7872
:104EC000E4B2651CEDB21D70022515551C78E4B2E4
:104ED000651CEDB21D7002AB1B791355754B187034
:104EE0007C4B186001F0D7F9012702AB9D78754B18
:104EF0001A781C00954211D1774A02A910780979D5
:104F00000130884209D01078744EC0B23070002948
:104F100003D0734E30683843306011701B789D4267
:104F200001D001F00AFC8021654AC90413680B43D3
:104F3000136002AB5B791100102B01D100F081FDF1
:104F400000D999E0072B00D1FEE14DD8032B00D109
:104F500055E13FD8012B00D10EE1022B01D001F029
:104F6000ECFB06200526584B1978C9B24A1CD2B270
:104F70001A70574A50541978C9B2481CC0B21870F8
:104F800056541978C9B2481CC0B218700020505449
:104F90001978C9B2481CC0B218704C48844665469E
:104FA0000078C0B2441CE4B22C7050541978C9B2D5
:104FB000481CC0B21870832050541978C9B2481CDC
:104FC000C0B2187056541978C9B2481CC0B21870D3
:104FD0000023EAE1052B00D157E100D906E3404A5E
:104FE000404B11680B404DE10B2B00D1B9E308D8C1
:104FF000092B01D101F061FB334A354900D82EE37A
:10500000DAE30E2B00D174E301D901F015FB0C2B70
:1050100001D001F092FB05202B4B2C4D1978C9B221
:105020004A1CD2B21A702A4A50541978C9B2481C84
:10503000C0B21870042050541978C9B2481CC0B2CC
:105040001870002050541978C9B2481CC0B21870AA
:105050002878C0B2441CE4B22C7050541978C9B2FC
:10506000481CC0B218708B2050541978C9B2481C23
:10507000C0B21870FF2398E1172B01D101F09CF901
:1050800032D8132B01D100F084FF09D8112B01D1A4
:1050900000F08FFD122B01D100F03EFD01F04DFB21
:1050A000152B01D101F03DFA01D801F06FFA01F0A2
:1050B000E4F8C04684070020910700207405002012
:1050C0006805002038040020E60200203C0500208E
:1050D0003B04002088070020630500208007002093
:1050E0007C070020FFFFFBFF302B01D100F008FC04
:1050F0000ED8192B00D16DE101D201F0B0F81A2BB6
:1051000001D001F01AFB02AB1A7AE24900234FE109
:10511000322B01D100F010FC00D27EE3712B01D0C4
:1051200001F00BFB0420DC4BDC4D1978C9B24A1CA2
:10513000D2B21A70DA4A50541978C9B2481CC0B2B7
:105140001870032050541978C9B2481CC0B21870A6
:10515000002050541978C9B2481CC0B21870287881
:10516000C0B2441CE4B22C7050541978C9B2481C27
:10517000C0B21870F12318E10625C7490C78E4B2D3
:10518000601CC0B20870C64805550C78E4B2651CB6
:10519000EDB20D70052505550D78EDB26C1CE4B22D
:1051A0000C70002444550D78EDB26E1CF6B20E70F2
:1051B00044550D78EDB26E1CF6B20E708126465540
:1051C0000D78EDB26E1CF6B20E70FE2646550D78C7
:1051D000EDB26E1CF6B20E70AF214155AF49B14829
:1051E0000B70B1490C70B1490C70016899430160B2
:1051F000AF4B1B78A34201D101F09FFA2CE00421B0
:105200008020AC4BC0021960A6490B6803430B60B9
:10521000A74B1B78002B1FD0A74B1B88C72B1BD875
:1052200080214024A54883680B438360A448836899
:10523000A34383600020A34B1870A34B0530187064
:10524000A24B19701168A24B0B401360FA22A14BBC
:1052500052001A6001F071FA80211368C90110E050
:10526000681EC0B22100FBF7E5FC072D01D001F05C
:1052700064FA3E2C01D001F060FA8021964A0905BB
:1052800013680B43136001F058FA0B20824B002582
:105290001978824EC9B24A1CD2B21A70804A505450
:1052A0001978C9B2481CC0B218700A205054197835
:1052B000C9B2481CC0B2187055541978C9B2481CFC
:1052C000C0B218703078C0B2441CE4B2347050548C
:1052D0001978C9B2481CC0B218708420505419788B
:1052E000C9B2481CC0B2187057541978C9B2481CCA
:1052F000C0B2187055541978C9B2481CC0B21870A1
:105300003E2050541978C9B2481CC0B21870734876
:105310000468240E54541C78E4B2611CC9B219709C
:105320000168090CC9B211551C78E4B2611CC9B2FC
:1053300019700168090AC9B211551978C9B24C1C13
:10534000E4B21C700368BBE20520534B534D19783F
:10535000C9B24A1CD2B21A70514A50541978C9B213
:10536000481CC0B21870042050541978C9B2481CA7
:10537000C0B21870002050541978C9B2481CC0B28D
:1053800018702878C0B2441CE4B22C7050541978BC
:10539000C9B2481CC0B21870822050541978C9B2E2
:1053A000481CC0B2187002AB9B79535401F0C5F988
:1053B000D8B2824205D902AC1819407AC8540133D8
:1053C000F6E700238B540421364A02ABDF711368E1
:1053D0000B43136002ABD979002900D180E0002390
:1053E0002C4AD15CD8B2002903D00133182BF8D154
:1053F0001800294BC41D1978E4B2C9B24A1CD2B2B4
:105400001A70274A54541978C9B24C1CE4B21C7063
:10541000841DE4B254541C78E4B2611CC9B2197002
:10542000002111551C78E4B2651CEDB21D701B4DB6
:10543000AC4661462D78EDB26E1CF6B20E70155575
:105440001C780021E4B2651CEDB21D709525155540
:105450001C78104EE4B2651CEDB21D701155002190
:105460001C78E4B2651CEDB21D7017551C78E4B2CF
:10547000651CEDB21D701055CCB2844201D301F011
:105480005CF91C78E4B2651CEDB21D70755C0131ED
:105490001555F1E74A050020E60200203C050020F2
:1054A0003B0400207C0700208007002063050020CB
:1054B0001203002000E100E07005002000400050D1
:1054C000C04000506E050020AC0200207205002094
:1054D000FFFFBFDFDC02002068050020B4020020CF
:1054E0001224F84BF84E1878C0B2421CD2B21A708F
:1054F000F64A14541878C0B2441CE4B21C7011244B
:1055000014541878C0B2441CE4B21C7011541878BA
:10551000C0B2441CE4B21C703478E4B2651CEDB235
:10552000357014541878C0B2441CE4B21C70952431
:1055300014541878C0B2441CE4B21C70115418788A
:10554000C0B2441CE4B21C7011541978C9B2481C92
:10555000C0B21870092050541978C9B2481CC0B2A2
:105560001870422050541978C9B24C1CE4B21C7017
:10557000692454541978C9B24D1CEDB21D704425EC
:1055800055541978C9B24D1CEDB21D705454197898
:10559000C9B24C1CE4B21C7050541978C9B2481CF2
:1055A000C0B218706F2050541978C9B24C1CE4B2C4
:1055B0001C7050541978C9B2481CC0B218707320BE
:1055C00050541978C9B2481CC0B218707420505495
:1055D0001978C9B2481CC0B21870652050541978A7
:1055E000C9B2481CC0B218707223DEE60720B54B62
:1055F00000251978B44EC9B24A1CD2B21A70B34A07
:1056000050541978C9B2481CC0B2187006205054C2
:105610001978C9B2481CC0B2187055541978C9B26B
:10562000481CC0B218703078C0B2441CE4B2347068
:1056300050541978C9B2481CC0B218708520505413
:105640001978C9B2481CC0B218700B205054197890
:10565000C9B2481CC0B21870575400F090FF8025A2
:105660009B4BAD021C689B482C4207D01D689A4C8E
:105670002C401C607F230478234005E01C682C43E9
:105680001C60802304782343037013788E4DDBB2B3
:10569000581CC0B210700520C8541378DBB2581CD7
:1056A000C0B210700420C8541378DBB2581CC0B2CA
:1056B00010700020C8541378DBB2581CC0B21070B0
:1056C0002878C0B2441CE4B22C70C8541378DBB202
:1056D000581CC0B210708720C8541078C0B2431C48
:1056E000DBB213707A4B1B685B0C3B400B5401F030
:1056F00024F80620734B00241978734EC9B24A1C53
:10570000D2B21A70714A50541978C9B2481CC0B24A
:105710001870052050541978C9B2481CC0B21870CE
:1057200054541978C9B2481CC0B218703078C0B24D
:10573000451CEDB2357050541978C9B2481CC0B23E
:105740001870862050541978C9B2481CC0B218701D
:1057500054541978C9B2481CC0B21870545400F09F
:10576000ECFF0520574B584D1978C9B24A1CD2B2EC
:105770001A70564A50541978C9B2481CC0B21870F1
:10578000042050541978C9B2481CC0B218700020C7
:1057900050541978C9B2481CC0B218702878C0B2E9
:1057A000441CE4B22C7050541978C9B2481CC0B2E1
:1057B0001870882000F038FF1378434DDBB2581C76
:1057C000C0B210700520C8541378DBB2581CC0B2A8
:1057D00010700420C8541378DBB2581CC0B210708B
:1057E0000020C8541378DBB2581CC0B2107028785F
:1057F000C0B2441CE4B22C70C8541378DBB2581CFD
:10580000C0B210708A20C8541378DBB2581CC0B2E2
:1058100010708022CA5400F090FF04212F4B304DAD
:105820001960304B1F70304B1B88C72B18D8402491
:105830002E487C3183680B4383602D488368A343E3
:10584000836000202B4B1870224B29707B39197014
:105850001168294B0B401360FA22284B52001A6042
:105860000520184B184E1978C9B24A1CD2B21A70CA
:10587000164A50541978C9B2481CC0B21870042096
:1058800050541978C9B2481CC0B218700020505446
:105890001978C9B2481CC0B218703078C0B2441C24
:1058A000E4B2347050541978C9B2481CC0B21870B0
:1058B000B02050541978C9B2481CC0B218702B7867
:1058C000DBB272E5E60200203C0500203B0400202C
:1058D0007C070020AC020020FFFFFDFF00E100E09C
:1058E0007205002062050020700500200040005075
:1058F000C04000506E050020FFFFBFDFDC0200202B
:105900008020CA498B6883438B60C94940388B68C3
:1059100003438B600023C7490B70C74908780528EB
:1059200001D1023000E006200870C4490B708121CB
:10593000136889050B4313600F20C14BC14D1978C3
:10594000C9B24A1CD2B21A70BF4A50541978C9B2AF
:10595000481CC0B21870042050541878C0B2411CC2
:10596000C9B21970002111541878C0B2441CE4B2B5
:105970001C702C78E4B2661CF6B22E7014541878A1
:10598000C0B2441CE4B21C70B02414541878C0B2E5
:10599000441CE4B21C70A94CA4462478E4B214540C
:1059A0001878C0B2441CE4B21C700924145418784E
:1059B000C0B2441CE4B21C7011541878C0B2441C2C
:1059C000E4B21C702C78E4B2661CF6B22E7014544B
:1059D0001878C0B2441CE4B21C70B2241454187875
:1059E000C0B2441CE4B21C7017541878C0B2441CF6
:1059F000E4B21C706446247864B28C4204DA9349A1
:105A00004C780A216143C9B211541978C9B2481CB3
:105A1000C0B21870002050541978C9B24C1CE4B2BE
:105A20001C7050541978C9B24C1CE4B21C7002248A
:105A300054541978C9B24C1CE4B21C70505400F094
:105A40007CFE834B1A687E4B520331D505201978B2
:105A50007C4DC9B24A1CD2B21A707B4A5054197894
:105A6000C9B2481CC0B21870042050541978C9B289
:105A7000481CC0B21870002050541978C9B2481C94
:105A8000C0B218702878C0B2441CE4B22C705054D4
:105A90001978C9B2481CC0B21870B0205054197897
:105AA000C9B2481CC0B2187064480078C0B25054E3
:105AB000052019780025C9B24A1CD2B21A70624A70
:105AC000604E50541978C9B2481CC0B218700420F6
:105AD00050541978C9B2481CC0B21870555419787E
:105AE000C9B2481CC0B218703078C0B2441CE4B2CD
:105AF000347050541978C9B2481CC0B21870922042
:105B000050541978C9B2481CC0B2187012235354AB
:105B1000504B1D7000F011FE02AB9B794D4A152BC6
:105B200037D013D8102B2CD007D80C2B3FD00F2BED
:105B300025D00B2B3DD10E233AE0122B25D022D3BA
:105B4000132B24D0142B34D1052331E01A2B26D06B
:105B500008D8172B21D01ED3182B26D0192B28D1CB
:105B60000D2325E0FC2B1ED003D81C2B21D11023A4
:105B70001EE0FD2B15D0FE2B1BD1112318E00023B6
:105B800016E0177015E0022312E0032310E004234F
:105B90000EE006230CE007230AE0082308E00923AF
:105BA00006E00A2304E00B2302E00C2300E00F23AD
:105BB000137006200525224B224E1978C9B24A1CC3
:105BC000D2B21A70204A50541978C9B2481CC0B2D7
:105BD000187055541978C9B2481CC0B2187000200A
:105BE00050541978C9B2481CC0B218703078C0B28D
:105BF000441CE4B23470174C50542178112900D958
:105C0000AFE1080001F002F8280036004C00610006
:105C100077008D00A300B100DE00F4000B0120012D
:105C2000350143015B0169017F019601004000508D
:105C3000C040005062050020AC0200207205002028
:105C4000E60200203C0500203B040020E702002083
:105C50007C070020640200201878C0B2451CEDB219
:105C60001D70902515541878C0B2451CEDB21D70FA
:105C70000F2522E01878C0B2451CEDB21D709025AA
:105C800015541878C0B2451CEDB21D70102515547E
:105C90001878C0B2451CEDB21D70E54B5B7847E14A
:105CA0001878C0B2451CEDB21D70902515541878B7
:105CB000C0B2451CEDB21D70112515541878C0B244
:105CC000451CEDB21D70175460E11878C0B2451C38
:105CD000EDB21D70902515541878C0B2451CEDB278
:105CE0001D70122515541878C0B2451CEDB21D70F8
:105CF000CF4B5B79E1E01878C0B2451CEDB21D7066
:105D0000902515541878C0B2451CEDB21D701325AE
:105D100015541878C0B2451CEDB21D70C44B9B7869
:105D200006E11878C0B2451CEDB21D7090251554DF
:105D30001878C0B2451CEDB21D70142515541878A2
:105D4000C0B2451CEDB21D70B94BDB78F0E018789D
:105D5000C0B2451CEDB21D70902515541878C0B224
:105D6000451CEDB21D701525A7E71878C0B2451C7B
:105D7000EDB21D70902515541878C0B2451CEDB2D7
:105D80001D7016251554AA480079C0B203280BD0FF
:105D9000042810D0022800D0F8E01878C0B2451CC2
:105DA000EDB21D708B23F0E01878C0B2451CEDB247
:105DB0001D709B23E9E01878C0B2451CEDB21D7040
:105DC000AA23E2E01878C0B2451CEDB21D70902500
:105DD00015541878C0B2451CEDB21D701725155426
:105DE0001878C0B2451CEDB21D70914B9B799FE0B5
:105DF0001878C0B2451CEDB21D7090251554187866
:105E0000C0B2451CEDB21D701A2515541878C0B2E9
:105E1000451CEDB21D70864B5B795B084DE0187830
:105E2000C0B2451CEDB21D70902515541878C0B253
:105E3000451CEDB21D70FD2515541878C0B2451CE7
:105E4000EDB21D700823A0E01878C0B2451CEDB279
:105E50001D70902515541878C0B2451CEDB21D7008
:105E6000FC2515541878C0B2451CEDB21D701823DE
:105E70008BE01878C0B2451CEDB21D70902515540A
:105E80001878C0B2451CEDB21D70182515E71878BA
:105E9000C0B2451CEDB21D70902515541878C0B2E3
:105EA000451CEDB21D70192515541878C0B2451C5B
:105EB000EDB21D705E4B5B799B093B4065E0187845
:105EC000C0B2451CEDB21D70902515541878C0B2B3
:105ED000451CEDB21D700B2539E01878C0B2451C89
:105EE000EDB21D70902515541878C0B2451CEDB266
:105EF0001D700C2515541878C0B2451CEDB21D70EC
:105F00004B4BDB7C14E01878C0B2451CEDB21D7021
:105F1000902515541878C0B2451CEDB21D701C2593
:105F200015541878C0B2451CEDB21D70404B9B7CD7
:105F3000DBB22AE01878C0B2451CEDB21D70902586
:105F400015541878C0B2451CEDB21D70FE251554CD
:105F50001878C0B2451CEDB21D70354B5B79DB097A
:105F600013E01878043815540425187803381554AC
:105F70001878C0B2451CEDB21D70912515541878E3
:105F8000C0B2451CEDB21D70FF23135401312170C6
:105F9000D3E3284C284D23780020DBB25A1CD2B220
:105FA00022700622EA542378244EDBB25A1CD2B265
:105FB00022700522EA542378DBB25A1CD2B2227036
:105FC000E8542378DBB25A1CD2B222703278D2B2B3
:105FD000511CC9B23170EA542378DBB25A1CD2B2D8
:105FE00022709022EA542278D2B2531CDBB2237082
:105FF00002AB9B79AB54142B5CD035D8102B00D15D
:10600000AEE01DD80B2B00D1E3E00C2B00D01EE13D
:1060100023781220DBB25A1CD2B2227002AAD479A1
:106020002100EC54FAF706FE014BDC7485E3C04610
:10603000E7020020E60200203B0400203C0500208F
:10604000122B24D0132B00D001E123780120DBB2E6
:106050005A1CD2B2227002AAD4792100EC54FAF769
:10606000E9FDDA4B9C7068E3192B00D198E004D865
:10607000162B35D0172B5DD0E9E01C2B00D1C1E0E9
:10608000FE2B00D1CDE01A2B00D0E0E076E0CF4E21
:1060900002AA7379D0792278DBB2D2B2511CC9B28C
:1060A0002170002802D0AF543B4301E0A854BB4309
:1060B0001C00A1E002ABDB79FA2B02D9FA2302AA79
:1060C000D37123780220DBB25A1CD2B2227002AA0A
:1060D000D4792100EC54FAF7ADFDBC4BDC702CE315
:1060E00002ABDB79B94EAA2B08D9AA2302AA042154
:1060F0000320D371FAF79EFD042312E09A2B08D8EF
:106100008B2302AA02210320D371FAF793FD022305
:1061100007E003219B2302AA0800D371FAF78AFD46
:10612000032333712378DBB25A1CD2B2227002AA45
:10613000D27992E002ABDB79632B02D8002302AA6A
:10614000D37123780520DBB25A1CD2B2227002AA86
:10615000D4792100EC54FAF76DFD9C4B9C71ECE274
:106160002378DBB25A1CD2B2227002AAD479210061
:10617000EC54FAF75FFD954B5C70DEE2934E02AA99
:106180007379D0792278DBB2D2B2511CC9B22170B6
:10619000002802D0AF54022429E0A854022216E0BD
:1061A0008A4E02AA7379D279DBB2002A07D022780C
:1061B000D2B2511CC9B22170AF54402417E02278EA
:1061C000D2B2511CC9B221700021A954402293437C
:1061D0006EE77E4E02AA7379D0792278DBB2D2B212
:1061E000511CC9B22170002803D08024AF541C4335
:1061F00002E07F24A8541C4021000420FAF71AFD75
:1062000074719AE223781120DBB25A1CD2B2227048
:1062100002AAD4792100EC54FAF70CFD6B4B9C7464
:106220008BE222780420D2B2531CDBB2237002AB83
:10623000DB79AB547F22654D6C7914405A1E934133
:10624000DB011C432100FAF7F5FC6C7175E2237841
:10625000DBB25A1CD2B222700022EA546DE202ABC9
:106260009A795B4B1A7002AAD2795A7002AA127AF2
:106270009A7002AA527ADA705FE202AB9A79092A1E
:1062800005D802A81318DB799C46092B08D90A689F
:10629000504B13400B600A684F4B13400B60D1E327
:1062A0004E4B1C78E4B2611CC9B21970614650189B
:1062B000C0B24B49851DEDB20D551C780530E4B2D6
:1062C000651CEDB2C0B21D7008551C78E4B2601CAC
:1062D000C0B21870002008551C784248E4B2651C12
:1062E000EDB21D703F4D2D78EDB26E1CF6B206700A
:1062F0000D551C780020E4B2651CEDB21D7093258D
:106300000D551C780090E4B2651CEDB21D700A5565
:106310001C0068460578AA420ED9257802A8EDB27D
:106320006E1CF6B22670009E3618F6792C4846553B
:10633000009801300090ECE71878C0B2451CEDB22F
:106340001D7063460B540023D9B28C450CD92178BB
:1063500002ADC9B2481CC0B2207098184019007A2A
:106360001F4D01336854EFE702ABDD790A210023AA
:10637000303DEDB20133D8B2824207D902AC4D4371
:106380001819C07930382D18EDB2F3E702A9531867
:106390000A2000211C7A303CE4B20131CBB29C458A
:1063A00001D8FEF75DFF8B1802AE44439B191B7AA0
:1063B000303BE418E4B2F0E702AB9979092913D92C
:1063C0001168044B0B40136038E3C046E70200201D
:1063D000E2020020FFFFFFFDFFFFFFFBE6020020BF
:1063E0003B0400203C05002000220A2002ABDB79A0
:1063F000303BDBB200930132D3B299420AD902ACEE
:106400001319DC79009D23004543303BEB18DBB2C8
:106410000093F0E7009B072B02D10B22E74BDA71C8
:106420000800E74C09302278C0B2D2B2531CDBB26C
:106430002370E44B98542278D2B2501CC0B2207022
:1064400008000830C0B298542078C0B2421CD2B2C2
:10645000227000221A542078C0B2451CEDB225707B
:10646000D94DAC4662462D789C46EDB26E1CF6B214
:1064700016701D5420780022C0B2451CEDB2257064
:10648000932526001D542078C0B2451CEDB225701E
:106490001954D0B288420BD2307802ABC0B2451C3E
:1064A000EDB23570D5186346ED7901321D54F0E731
:1064B0002378C44DDBB25A1CD2B222700322EA54B4
:1064C0002678009AF6B2731CDBB22370BB4B6421B2
:1064D000985CC0B200F0A4FB3030009AB74BC0B259
:1064E000A855985C6421C0B200F020FC2678CBB29D
:1064F000F6B20093731CDBB223700A21009800F0FF
:106500008FFB3030C0B2A85526780A21F6B2731C32
:10651000DBB22370009800F009FC3031C9B2A955F4
:106520000BE105201168A94B00250B401360A44B1B
:10653000A54E1978C9B24A1CD2B21A70A14A505459
:106540001978C9B2481CC0B2187004205054197888
:10655000C9B2481CC0B2187055541978C9B2481C49
:10656000C0B218703078C0B2441CE4B234705054D9
:106570001978C9B2481CC0B21870942050541978C8
:10658000C9B2481CC0B218705554D6E0904802A950
:106590000368497A1B0E994200D0CEE002AB9C7A88
:1065A000FF230168090C19408C4200D0C5E0016846
:1065B00002ACE47A090A19408C4200D0BDE002A97D
:1065C0000068097B0340994200D0B6E08021052095
:1065D000136889040B431360794B7B4D1978C9B25A
:1065E0004A1CD2B21A70774A50541978C9B2481C62
:1065F000C0B21870042050541978C9B2481CC0B2F7
:106600001870002050541978C9B2481CC0B21870D4
:106610002878C0B2441CE4B22C7050541978C9B226
:10662000481CC0B21870942050541978C9B2481C44
:10663000C0B21870575480E002AB9B79002B7CD11C
:1066400002AB5B7A3E2B78D1614902AA0B68927A41
:106650001B0E9A4271D102ABD87AFF230A68120C42
:106660001A40904269D10A6802A8007B120A1A40B7
:10667000904262D102AA0968527B0B409A425CD1D7
:10668000FAF7CAFAFAF7B0FAF8204002FAF782FAF3
:106690002378504A504C1B021343236021684F4813
:1066A000FAF71EFA03214E4A13680B43236023684E
:1066B00013604C4A4C4B1A60FEE780204B498B68B4
:1066C00083438B604A4940388B6803438B60FA21CF
:1066D000484B8900198000218120474B80051970A3
:1066E000136803431360454A454B106803409020EC
:1066F0001360444A9368034393608022424B9201A3
:10670000DA67424B424A1970424BFF311A60424AE3
:1067100011701A68002AFCD12B4B1A70FAF77CFA18
:1067200003212F4A13680B4313602E4A2E4B1A6025
:10673000A022D20593683B43936002AB9B78002B69
:1067400000D063E102AA1279092A00D1F9E00AD83F
:10675000032A00D12CE1042A00D057E1274A284B14
:1067600011680B4051E1302A00D19BE0312A00D062
:106770004CE10421294A204C1160294A1770294A0A
:106780001188294AC72957D880204026174DA96863
:106790000143A960164DA968B143A96023490B7054
:1067A0000521234B197020701168224B0B40136098
:1067B000FA22184B52001A6043E0C046E70200205C
:1067C000E60200203B0400203C050020FFFFFFFD07
:1067D000B40200203E00FFFFCC0200201CF00100AC
:1067E00000C000500400FA050CED00E0004000502D
:1067F000C0400050E0020020720500207C0700200D
:10680000FFFFFBFF8040005004E100E09007002004
:10681000DC050000DC0200203904002000E100E07B
:106820006205002070050020680500206E0500202C
:10683000AC020020FFFFBFDF80211368C9010B43BA
:1068400013600520804B814E1978C9B24A1CD2B220
:106850001A707F4A50541978C9B2481CC0B21870D7
:10686000042050541978C9B2481CC0B218700020D6
:1068700050541978C9B2481CC0B218703078C0B2F0
:10688000451CEDB2357050541978C9B2481CC0B2DD
:106890001870B02050541978C9B2481CC0B2187092
:1068A00023784BE080206B498A6882438A606A497A
:1068B00040388A6802438A60684A1370684B1A78C5
:1068C000052A01D1023200E00622002081210524A0
:1068D000644D1A70644A2870136889050B4313606D
:1068E000594B5A4E1978C9B24A1CD2B21A70584A3A
:1068F00054541978C9B24C1CE4B21C70042454548A
:106900001978C9B24C1CE4B21C7050541978C9B241
:10691000481CC0B218703078C0B2441CE4B2347065
:1069200050541978C9B2481CC0B21870B0205054E5
:106930001978C9B2481CC0B218702B78DBB2535416
:1069400064E0802043498A6882438A604249403833
:106950008A6802438A60FA218120444A89001180B2
:10696000404A414913700A68800502430A60802149
:106970003F4A8901D167FF213E4A13703E4A3F4B8F
:106980001A603F4A11701A68002AFCD12F4B1A7006
:10699000FAF742F903213B4A13680B4313603A4A62
:1069A0003A4B1A60A022D20593683B4393602DE0D6
:1069B00080203749C0020A6802430A60354A1178CC
:1069C000294A00291DD034490988C72919D88020AF
:1069D0004025204CA1680143A1601F4CA168A94338
:1069E000A1602E490B7005211D4B19701D4B1870AD
:1069F00011682B4B0B401360FA22204B52001A6097
:106A000004E080211368C9010B43136002AB1A78BC
:106A10005B7801339A4210DDDBB2D21A02A90A7008
:106A2000002201320198D1B2884201D8FEF75DFA06
:106A300002A81918895C8154F3E70B4A1168194BB5
:106A40000B40136013B0F0BDE60200203C050020AF
:106A50003B04002000400050C04000506205002070
:106A6000AC0200207205002068050020E002002032
:106A700004E100E090070020DC050000DC020020BB
:106A80003904002000C000500400FA050CED00E0BD
:106A90007C07002012030020700500206E050020F6
:106AA000FFFFBFDFFFFFFFFBF7B59C4608AB1D787C
:106AB000A02380260192DB05DC6876053443DC6088
:106AC000DF68224C2D043C40DC60214C03276369C5
:106AD0001A0063463B409F000C239A4317436761AB
:106AE000A7691C4B3B402B430125A361A36833439B
:106AF000A360194B1C6A2C431C62002803D11C6A3A
:106B00001648204003E08024186AE40020431862FD
:106B10000C20002902D1196A814305E0012905D121
:106B2000196A814304200143196208E0022903D154
:106B3000196A81430820F6E7196A08431862FF20A2
:106B4000596A019A81430A435A62F7BDFFFFFFEF7A
:106B500000020050FFFF00FF00000E40FFFBFFFFA0
:106B600010B5194C236BDB070CD5184A1368002BA2
:106B700001D0506898470721154A13688B4306399E
:106B80000B431360236B9B070CD5104A1369002B32
:106B900001D09068984707210D4A13688B43053947
:106BA0000B431360236B5B070CD5084A5369002B1A
:106BB00001D0D06898470721054A13688B430339F1
:106BC0000B43136010BDC04600000E408802002039
:106BD00030000E400721064A13688B4306390B43E9
:106BE00080211360034A0901136A0B431362704743
:106BF00030000E4000000E4002B4714649084900C2
:106C0000095C49008E4402BC7047C04603B471461B
:106C1000490840004900095A49008E4403BC7047A6
:106C2000002243088B4274D303098B425FD3030ACB
:106C30008B4244D3030B8B4228D3030C8B420DD3DE
:106C4000FF22090212BA030C8B4202D3121209026C
:106C500065D0030B8B4219D300E0090AC30B8B42AA
:106C600001D3CB03C01A5241830B8B4201D38B0358
:106C7000C01A5241430B8B4201D34B03C01A5241FD
:106C8000030B8B4201D30B03C01A5241C30A8B4240
:106C900001D3CB02C01A5241830A8B4201D38B022B
:106CA000C01A5241430A8B4201D34B02C01A5241CF
:106CB000030A8B4201D30B02C01A5241CDD2C30941
:106CC0008B4201D3CB01C01A524183098B4201D3BD
:106CD0008B01C01A524143098B4201D34B01C01AA8
:106CE000524103098B4201D30B01C01A5241C30820
:106CF0008B4201D3CB00C01A524183088B4201D38F
:106D00008B00C01A524143088B4201D34B00C01A7A
:106D10005241411A00D20146524110467047FFE7E6
:106D200001B5002000F0F0F802BDC0460029F7D000
:106D300076E7704703460B437FD4002243088B421B
:106D400074D303098B425FD3030A8B4244D3030BF2
:106D50008B4228D3030C8B420DD3FF22090212BAB7
:106D6000030C8B4202D31212090265D0030B8B4233
:106D700019D300E0090AC30B8B4201D3CB03C01A1D
:106D80005241830B8B4201D38B03C01A5241430BF8
:106D90008B4201D34B03C01A5241030B8B4201D3E8
:106DA0000B03C01A5241C30A8B4201D3CB02C01A53
:106DB0005241830A8B4201D38B02C01A5241430ACB
:106DC0008B4201D34B02C01A5241030A8B4201D3BA
:106DD0000B02C01A5241CDD2C3098B4201D3CB0161
:106DE000C01A524183098B4201D38B01C01A524110
:106DF00043098B4201D34B01C01A524103098B4214
:106E000001D30B01C01A5241C3088B4201D3CB00FE
:106E1000C01A524183088B4201D38B00C01A5241E1
:106E200043088B4201D34B00C01A5241411A00D291
:106E300001465241104670475DE0CA0F00D04942FA
:106E4000031000D34042534000229C4603098B426A
:106E50002DD3030A8B4212D3FC22890112BA030AF2
:106E60008B420CD3890192118B4208D38901921174
:106E70008B4204D389013AD0921100E08909C309F9
:106E80008B4201D3CB01C01A524183098B4201D3FB
:106E90008B01C01A524143098B4201D34B01C01AE6
:106EA000524103098B4201D30B01C01A5241C3085E
:106EB0008B4201D3CB00C01A524183088B4201D3CD
:106EC0008B00C01A5241D9D243088B4201D34B00E8
:106ED000C01A5241411A00D20146634652415B102A
:106EE000104601D34042002B00D54942704763460B
:106EF0005B1000D3404201B5002000F005F802BD50
:106F00000029F8D016E770477047C046000000001F
:106F100020000000000010002000100030353A3F33
:106F200044494E54585C61666B7075A512646403E5
:106F300081C80B3E041EFFFFFFFFFFFFFF0530FF70
:106F4000020408100100000002000000020000001E
:046F50000400000039
:106F5400FF4040404040404033404040344035369C
:106F640040404040404040403A4040403B403C3735
:106F7400404040403F403D3840403E3940FB404067
:106F84004040404040404040244040402340222173
:106F9400404040401F401E2040401D1C401B4040BC
:106FA400404040401940181A4040171640154040D0
:106FB400404025144013404040324040404040404F
:106FC4004040404040404040FE4040400E400D0C98
:106FD400404040400A40090B4040080740064040FA
:106FE400404040400440030540400201400040400E
:106FF40040400F104011404040124040404040404B
:1070040040404040FD402B3040402A2F403140401A
:107014004040292E402D4040402C404040404040BC
:107024004040FA28402740404026404040404040ED
:1070340040FC0000001BB70000000000008051016C
:10704400102700000080510100805101160000004B
:00000001FF
